:020000040000FA
:06000000C9EF35F012000B
:06000800B9EF31F0120017
:06001800C7EF31F01200F9
:06002A0003001D6C000044
:100030008000000068000000136C00006E0F0000DC
:100040000A0000000E6C0000FA030000050000002A
:100050000101D86BD96B0301326B00018F6B120069
:10006000A4EC10F0DF6A00019051020A59E0030A83
:100070001CE0010A65E191EC2AF0000963E10E0140
:100080005D5160E05D51E66EE66A5E0EE66E0E0E54
:10009000E66E03EC2BF0E8EC0EF00001010E906F21
:1000A000D7DF0E01640E3E6F4DD095EC2AF00009AB
:1000B00033E00001020E906F0E015D29156AE850D1
:1000C00000018D5F15508E5B0E015D51146E156A37
:1000D000960ED8801456000E15561406155A14C0E4
:1000E000E6FF15C0E6FF5D51176A5D0F166E0E0E36
:1000F0001722010E1626000E172216C0E6FF17C0A3
:10010000E6FF5D0EE66E0E0EE66EABEC2BF0186EA3
:10011000060EE15E185016D00E013E5113E110D0CC
:100120000101D8510AE0D8C1D9F1D851020802E240
:100130000E015D6B0001906B05D00E013E5102E196
:10014000010EDF6EDF5008E00101D9690E015D6B21
:100150000001906B30EC2BF0E552CCEF0EF091ECFF
:100160002AF0000906E10001905103E10E015D5102
:1001700001E0010C000CD0EC0EF0FC0EDB50000195
:10018000156A8D25146E8E511522010E1426000E4F
:100190001522F30E145C0E0E15581CE2FC0EDB50FB
:1001A00052EC11F0EF6EFC0EDBCFE6FFE66AFAECE4
:1001B0000EF0010E2DEC10F080EC2BF0166E060EFA
:1001C000E15E1650FC0EDB28146E156AE850E4EC74
:1001D0000FF001D0010ECCEF0EF0D0EC0EF0020EBD
:1001E0000001176A8D25166E8E51172216C0E6FF84
:1001F00017C0E6FFFAEC0EF031EC2CF031EC11F008
:10020000E7CF17F0E552E7CF16F01650F324146E3F
:100210001750F420156EF30E145C0E0E15581BE2E9
:1002200035EC11F0010EF32452EC11F0EF6EFAEC04
:100230000EF0010E00012DEC10F0F7EC2BF0E8ECC5
:100240000EF035EC11F0020E1426000E152214509B
:10025000E4EC0FF001D0010ECCEF0EF0D0EC0EF07C
:100260000101C651040A49E0050A02E0030A43E11C
:10027000D85141E195EC2AF000093DE000018F5191
:1002800007E1FE0EDB50FE0803E00101E26B33D014
:1002900053EC10F009E2ECEC0FF0020E8F5D07E179
:1002A000FE0EDB50FE0803E00101D86924D00101F5
:1002B000E25102E1010EE26FFE0EDB50FD0869E142
:1002C000020E00018F5DEA6A320FE96E030EEA2228
:1002D000EF50FF0A0AE0050A05E0010A09E1010101
:1002E000010E08D00101040E05D00101050E02D057
:1002F0000101020ED86F000E4DD0D85148E195ECA7
:100300002AF0000944E0FE0EDB502E0803E1010153
:10031000010E08D00101E20507E1FE0EDB500D08D9
:1003200003E1020EE26F35D0020EE25D0EE1FE0E39
:10033000DB500A080AE1E26B00018F5103E0010182
:10034000020E18D00101010E15D079EC10F031EC3D
:1003500035F018EC10F0F350F4100EE179EC10F0D9
:1003600043EC35F0E552E552F350F41005E101019C
:10037000E26B040ED86F0DD0000153EC10F004E3D3
:100380000101E26BD86905D0ECEC0FF002D001015D
:10039000E26B000ECCEF0EF035EC2BF012EC2BF0F4
:1003A0005FDE0101D95112000E013E5102E1640EDF
:1003B0003E6F0E013E5103E0EFDF0009FAE001015C
:1003C000D95105E10E013E5102E10101D969010156
:1003D000D951020802E2D9511200000CA4EC10F02D
:1003E0000101C60503E0020EC65D04E1DF6A010EED
:1003F000D96F45D0FE0EDBCFC6F1CFEC29F0FE0E53
:10040000DB50020A19E0030A36E10001FE0EE16F3B
:10041000E26F580EE36FE00EE46F800EE66E250E7D
:10042000CAEC10F05FEC10F003E11C0E94EC10F03D
:10043000DF5025E1E66A1BD00001FE0EE16FE26F9E
:10044000280EE36FE00EE46FB00EE66E040ECAEC09
:1004500010F05FEC10F007E1100EE66E270EE66E6E
:10046000E66A5CEC11F0DF500AE1010EE66E37EC53
:1004700007F0E55203D0050E0101D96FDF6EDF50A2
:1004800002E00101C66BDF50E552CCEF0EF0A4ECA8
:1004900010F0DF6AF80EDB50DF5C38E2F90EDBCFDC
:1004A00006F0FA0EDBCF07F0FB0EDBCF08F0FC0EF8
:1004B000DBCF09F00A0E0B6E0C6A0D6A0E6A58EC5F
:1004C00035F00250E66E4AEC0FF0E552E750EF6E61
:1004D000FFEC0EF0B6EC0FF00A0E0B6E0C6A18EC87
:1004E0000FF058EC35F078EC0FF0040ED89014367D
:1004F000153616361736E806F9E14AEC0FF01450B7
:10050000EF26FFEC0EF0020EDF26C4D7E552CCEF4B
:100510000EF006EC11F0DE6ADE6ADE6ADD6ADD529C
:10052000DD52FC0EDB5010E0FC0EDB06EBEC0EF0B7
:10053000EF380F0BA4EC0FF0DD52DD52EBEC0EF0B8
:10054000EF50A4EC0FF0EBD7F7EC0FF0050EE15CE9
:1005500002E2E16AE552E16ECCEF0EF00AEC11F036
:10056000050EE76F0A0EE66E91EC10F065EC10F0E8
:10057000146E070EE15E14500101FD0EED6F0B0EBF
:10058000C2EC0EF0CCEF0EF00AEC11F0060EE76FA5
:10059000FE0EDB50030A0FE0010A0BE0030A07E03E
:1005A000010A03E0030ED96F0AD0050E05D0020E32
:1005B00003D0E86B02D0010EE86F01EC11F0CCEF34
:1005C0000EF00AEC11F00D0EE76FE150FD0FD5ECC7
:1005D00010F00F0ED880EE54270EED5403E2030EF8
:1005E000D96F1FD0080EE66E1FEC10F0166A176A5E
:1005F0000A0E0B6E0C6A3AEC11F002C0E6FF03C063
:10060000E6FF04C0E6FF05C0E6FF65EC10F0186EDB
:10061000070EE15E18500101FD0EEC6F0A0EC2ECF0
:100620000EF0CCEF0EF0A4EC10F0DEEC0EF00F0E9E
:10063000E76FDF6AFE0EDB50050A14E0070A0FE0E1
:10064000060A0DE0050A09E0020A07E0030A03E0D2
:10065000030ED96F0DD0100E03D0110E01D0120E63
:10066000E86F04D0010ED96F000E02D001EC11F03A
:10067000E552CCEF0EF0DEEC0EF0080E9BEF10F022
:100680000AEC11F0080EE76F1FEC10F00A0E0D6E69
:100690000E6A14C008F015C009F0B3EC35F004C0C0
:1006A00014F005C015F03FEC11F00A0E0D6E0E6A45
:1006B00016C008F017C009F0B3EC35F008C016F00A
:1006C00009C017F00A0E0D6E0E6AB3EC35F004C0C7
:1006D00016F005C017F0040ED89016361736E80449
:1006E000FBE1145016240101E86F01EC11F0CCEF8E
:1006F0000EF0DEEC0EF0070E9BEF10F0DEEC0EF0CD
:10070000090E9BEF10F0DEEC0EF00A0E9BEF10F0DE
:10071000A4EC10F0DEEC0EF0030E9BEC10F0DF6E9C
:10072000DF5022E1020E0101D95D1CE1030E03013D
:10073000365D18E1050EE66E370EE66E030EE66EC8
:10074000E8DE31EC11F006C0CBF107C0CCF108C0F7
:10075000CDF109C0CEF10EEC0FF046EC11F01EEC1D
:1007600011F002D0030EDF6EDF50E552CCEF0EF039
:10077000DEEC0EF06BEC10F0010EE96F080EC2EF2C
:100780000EF0DEEC0EF06BEC10F0E96B080EC2EF31
:100790000EF0A4EC10F0030E0101C65D04E1DF6A67
:1007A000010ED96F25D0030EC66FE6EC29F0949C9C
:1007B0009694949E0001E551E8B0828EE8A0829E56
:1007C000E651E8B08484E8A08494E751E8B0828CD4
:1007D000E8A0829C01012B0EFA6F020EF96F580EF1
:1007E00094EC10F0DF5004E1E66A41DBE552DF6E85
:1007F000DF50E552CCEF0EF0D9CFE6FFE1CFD9FFC5
:10080000020EE1263F0E0101FA170001E55107E053
:100810000101FA1DE76E010EE7CFDBFF03D0010EE9
:10082000FAC1DBFF010EDF6EDF5014E0010EDB507A
:10083000DF1402E0828E01D0829E0001E65104E0C6
:1008400084940000848403D0848400008494DF9E18
:10085000DF46EAD70001E55107E00101F91DE76E27
:10086000010EE7CFDBFF03D0010EF9C1DBFF010E64
:10087000DF6EDFB614D0010EDB50DF1402E0828E93
:1008800001D0829E0001E65104E08494000084843B
:1008900003D0848400008494DF9EDF46EAD7000101
:1008A000E55107E00101F71DE76E010EE7CFDBFF21
:1008B00003D0010EF7C1DBFF080EDF6EDF5014E03E
:1008C000010EDB50DF1402E0828E01D0829E000117
:1008D000E65104E084940000848403D08484000002
:1008E0008494DF9EDF46EAD70001E55107E001016D
:1008F000F81DE76E010EE7CFDBFF03D0010EF8C154
:10090000DBFF010EDF6EDF5014E0010EDB50DF1461
:1009100002E0828E01D0829E0001E65104E08494C0
:100920000000848403D0848400008494DF9EDF462A
:10093000EAD70001E75104E0829C0000828C03D0DA
:10094000828C0000829C000E00D0146E020EE15CCE
:1009500002E2E16AE552E16E1450E552E7CFD9FFB9
:100960001200D0EC0EF0030EE126060EE66EC3EC8C
:100970000FF057EC11F018EC0FF058EC35F006C002
:1009800014F007C015F008C016F009C017F006C033
:10099000E6FF07C0E6FF08C0E6FF09C0E6FFDAECA5
:1009A00010F075DD186E070EE15E1850010EDBCFFA
:1009B000F8F1F00EDF140101F76F0F0EDF14146E63
:1009C000050E145C01E3F7879CEC0FF0000E146E2B
:1009D000030EE15C02E2E16AE552E16E1450CCEFF5
:1009E0000EF0D9CFE6FF000ECCEF0EF0D9CFE6FF28
:1009F000000ECCEF0EF00DEC11F00DE0210E26EC08
:100A000010F009E2FE0EDB041F0B0101FA6F9CECF3
:100A10000FF0000E03D00101030ED96FCCEF0EF0E2
:100A20000101FA9B9CEC0FF0000C0101FA8B9CEC8D
:100A30000FF0000C0DEC11F0020805E2020EF36E4F
:100A4000FE0EF3CFDBFFFE0EDBCFF9F19CEC0FF0D7
:100A5000000ECCEF0EF00DEC11F004E11EEC11F0E5
:100A6000000E03D00101030ED96FCCEF0EF0A4EC01
:100A700010F0040E0101C65D04E1DF6A010ED96FBA
:100A800017D0040EC66FCFEC29F0E66A4B0ECAEC05
:100A900010F09D889D8A1C0E94EC10F0DF5004E14C
:100AA000E66AD4EC0DF0E552DF5002E00101C66BBE
:100AB000DF50E552CCEF0EF0D0EC0EF00E0EE1263A
:100AC000ADEC10F0B10EEE54080EEE54190EEE54CB
:100AD00007E2DE6AB10EDE6E080EDE6E190E17D06A
:100AE000ADEC10F03B0EEE54580EEE54080EEE54E2
:100AF00007E2DE6A3B0EDE6E580EDE6E080E07D091
:100B0000800EDE6EBA0EDE6E8C0EDE6E010EDD6EB7
:100B1000DD52DD52CBEC0FF0D9CFE9FF4EEC0FF0F8
:100B2000FB0E14C0DBFFFC0E15C0DBFFFD0E16C074
:100B3000DBFFFE0E17C0DBFF91EC10F0300EE66E0F
:100B40006B0EE66E000E22EC11F0E15E14503AECF2
:100B50000FF0A7EC10F0E76E0D0EE7CFDBFFDB50D8
:100B600054E1020E0101D95D50E100018F514DE0C9
:100B70005D0EE66E320EE66E030EE66EB8EC2CF0FD
:100B800031EC11F00B0EF3CFDBFF0C0EF4CFDBFFDB
:100B9000F3CF14F0F4CF15F0F350F41006E00B0E81
:100BA000DB2A0C0E0BE3DB2A09D0D9500B0FE96EC0
:100BB000DACFEAFF320EEE6E030EED6E0B0EDBCFD8
:100BC000E6FF0C0EDBCFE6FF0EEC31F0E552E5520E
:100BD000FB0E06C0DBFFFC0E07C0DBFFFD0E08C0EE
:100BE000DBFFFE0E09C0DBFFC3EC0FF011EC11F0D0
:100BF000EE5014240101CB6FEE501520CC6FEE5057
:100C00001620CD6FEE501720CE6F0D0EDB50146EF8
:100C10000E0EE15C02E2E16AE552E16E1450CCEFA7
:100C20000EF0D0EC0EF00E0EE126FE0EDB50030AA5
:100C300021E0070A1FE0060A10E0030A08E0010AA3
:100C400063E12D0EE66E6B0EE66E000E0BD02A0EE3
:100C5000E66E6B0EE66E000E05D0270EE66E6B0E8E
:100C6000E66E000EE66E3AEC0FF018EC2CF0146E07
:100C7000050E48D0D880000E0101CF55B10ED055D9
:100C8000080ED155190ED25508E281EC0FF0B10EC5
:100C9000155E080E165A190E11D0D880000ECF55C9
:100CA0003B0ED055580ED155080ED2550CE281ECB2
:100CB0000FF03B0E155E580E165A080E175A14C048
:100CC000DFFF010E0CD081EC0FF0800E145EBA0E27
:100CD000155A8C0E165A010E175A14C0DFFF15C094
:100CE000DBFF020E16C0DBFF030E17C0DBFF11ECAB
:100CF00011F0D5EC0EF01F0EE66E6B0EE66E000ED8
:100D000022EC11F0E15E14503AEC0FF0A7EC10F079
:100D1000146E0E0EE15C02E2E16AE552E16E1450DF
:100D2000CCEF0EF0D0EC0EF0030E0101D35D03E02A
:100D3000040ED35D04E17EEC10F0E55201D0000E0C
:100D4000CCEF0EF016EC11F0240E26EC10F011E2B0
:100D500079EC10F01A0EE66E6B0EE66E000EE66E83
:100D6000DAEC10F012EC34F0146E070E61EC11F0B6
:100D700003D00101030ED96F146E040EE15C02E290
:100D8000E16AE552E16E1450CCEF0EF01EEC11F06A
:100D9000000C16EC11F0160EE66E6B0EE66E000EF1
:100DA0001CEC0FF002E2E16AE552E16E1450CCEF68
:100DB0000EF016EC11F0FE0EDB50000806E2130EEA
:100DC000E66E6B0EE66E000E05D0100EE66E6B0E34
:100DD000E66E000E1CEC0FF002E2E16AE552E16EF5
:100DE0001450CCEF0EF00DEC11F004E11EEC11F0FC
:100DF000000E03D00101030ED96FCCEF0EF0CFEC43
:100E000029F01EEC11F0C66B000CCFEC29F01EECA3
:100E100011F000018B6B0101630EC66F000CA4EC96
:100E200010F0FE0EDB50630A16E0670A12E0070AB4
:100E30000EE0020A06E0030A04E0020A0FE1DFDF27
:100E40000BD0EEEC10F0EEEC01F0E55205D0A1DC99
:100E500003D00DDE01D0D9DFDF6E05D0030EDF6ECB
:100E60000101D96FC66BDF50E552CCEF0EF066EC96
:100E700011F01CE0670A14E0070A0EE0020A07E01E
:100E8000030A05E0020A15E146EC0FF014D0EEEC7F
:100E900010F0C4EC02F007D0EEEC10F0DCDD03D073
:100EA000EEEC10F0A0DFE552DF6E05D0A0EC0FF005
:100EB00002D0DF68D969DF50E552CCEF0EF006ECC6
:100EC00011F0FD0EDBCF06F0FE0EDBCF07F0086A57
:100ED000096A400E0B6E420E0C6E0F0E0D6E27EC63
:100EE0000FF00DE0030A0BE0010A09E0070A07E032
:100EF000670A05E0630A06E146EC0FF005D087ECCF
:100F000010F002D0DF68D96982EC10F002E2E16AE9
:100F1000E552E16E1450CCEF0EF006EC11F0FB0E32
:100F2000DBCF06F0FC0EDBCF07F0FD0EDBCF08F0C9
:100F3000FE0EDBCF09F057EC11F00D6A27EC0FF035
:100F40000DE0030A0BE0010A09E0070A07E0670A5F
:100F500005E0630A06E146EC0FF005D087EC10F0DF
:100F600002D0DF68D96982EC10F002E2E16AE55252
:100F7000E16E1450CCEF0EF006EC11F01FEC10F007
:100F8000166A176A57EC11F03AEC11F0C70EE96EC9
:100F9000010EEA6E8AEC0FF0010E14C0DBFF020EA8
:100FA00015C0DBFF030E16C0DBFF040E17C0DBFF0E
:100FB0000101C651010A0DE0030A0BE0010A09E034
:100FC000070A07E0670A05E0630A06E146EC0FF04E
:100FD00005D087EC10F002D0DF68D96982EC10F000
:100FE00002E2E16AE552E16E1450CCEF0EF0D0EC73
:100FF0000EF0070EE126020EDB68010EF36E030E03
:10100000F3CFDBFF040EDB6A050EDB6A060EDB6A3C
:10101000DF6ADFCF14F0156A166A030ED890143613
:1010200015361636E806FAE1D8EC0FF01424F36E04
:10103000EE501520F46EEE5016200DEC10F0090065
:10104000F5500900F5100900F5100800F51001E150
:1010500091D0F40EDBCF14F0F50EDBCF15F0F60EC9
:10106000DBCF16F0F70EDBCF17F0DFCF18F0196AE1
:101070001A6A030ED890183619361A36E806FAE1BD
:10108000D8EC0FF01824F36EEE501920F46EEE50E9
:101090001A20F86EF4CFF7FFF3CFF6FF0900F550F2
:1010A000145C0900F55015580900F5501658090050
:1010B000F55017585DE3F40EDBCF1BF0F50EDBCFD8
:1010C0001CF0F60EDBCF1DF0F70EDBCF1EF0DFCFEE
:1010D0001FF0206A216A030ED8901F362036213671
:1010E000E806FAE1D8EC0FF01F24F36EEE50202052
:1010F000F46EEE5021200DEC10F01B500900F55C51
:101100001C500900F5581D500900F5581E500900E3
:10111000F5582EE3030EDBCF22F0040EDBCF23F0D5
:10112000050EDBCF24F0060EDBCF25F0D950F80FEB
:10113000D5EC10F0EE502216EE502316EE50241689
:10114000EE502516225023102410251011E0020E17
:10115000DFCFDBFFD950030FE96EDACFEAFFD8907B
:10116000EF36010EEB36020EEB36030EEB3602D0F5
:10117000DF2A4FD7020EDB50146E070EE15C02E24D
:10118000E16AE552E16E1450CCEF0EF0D0EC0EF0B7
:10119000020EE126010EDB68DF6A5DEC0FF0EECF98
:1011A00014F0EECF15F0EECF16F0EFCF17F014508D
:1011B00015101610171017E0B6EC0FF05DEC0FF0DD
:1011C0001450EE180EE11550EE180BE11650EE1803
:1011D00008E11750EE1805E104E1010EDFCFDBFF57
:1011E00002D0DF2ADAD7010EDB50146E020EE15C6A
:1011F00002E2E16AE552E16E1450CCEF0EF0A4EC8D
:1012000010F0DF6A91EC10F083C0E6FF84C0E6FFC7
:1012100085C0E6FF86C0E6FF8E0EE66E5E0EE66EC9
:10122000000EDDEC0FF005E1000E151802E1000ED6
:10123000DF8091EC10F087C0E6FF88C0E6FF89C030
:10124000E6FF8AC0E6FF8E0EE66E5F0EE66E000ECB
:10125000DDEC0FF002E1000E151801E0DF8291ECE9
:1012600010F0910EE66E000EE66E90DF166E060E22
:101270004BEC11F002E1000E151801E0DF84DF50A5
:10128000E552CCEF0EF016EC11F0BEEC0EF037ECA0
:1012900010F011E3E3EC10F0A00EEE542F0EEE541C
:1012A000C50EEE54010EEE5406E3A00EDE6E860E61
:1012B000DE6E010E97D0BEEC0EF0C00EEE5C320E6C
:1012C000EE580A0EEE58030EEE581BE3E3EC10F056
:1012D000800EEE54F90EEE54370EEE54030EEE541B
:1012E00010E3040E0101C65D06E0200EDE6EA10EC5
:1012F000DE6E070E77D0400EDE6E420EDE6E0F0EF3
:1013000071D0D1EC10F0440EEE58950EB2EC0FF007
:101310000FE3ADEC10F04D0EEE54D20EEE54080E6D
:10132000EE5406E3C00EDE6E270EDE6E090E5AD0B6
:10133000DFEC10F0730EEE583B0EEE580D0EEE582B
:1013400010E3E3EC10F0400EEE543A0EEE54690E4A
:10135000EE540D0EEE5405E3DE6A6A0EDE6E180ED4
:1013600041D0D1EC10F0B10EB2EC0FF0190EEE58E6
:1013700011E3E3EC10F0800EEE54740EEE54D20E36
:10138000EE541A0EEE5406E3400EDE6E4B0EDE6E89
:101390004C0E28D0DFEC10F06D0EEE58C30EEE5858
:1013A000350EEE5809E3ADEC10F0280EEE54500E59
:1013B000EE54370EEE5412E2D1EC10F0E60EEE5879
:1013C000E80EEE58490EEE580FE3ADEC10F06D0E3E
:1013D000EE547C0EEE544D0EEE5406E3DE6A1B0E08
:1013E000DE6EB70EDE6E03D0DE6ADE6ADE6ADD6AAE
:1013F000DD52DD52F7EC0FF0040EE15C02E2E16A2F
:10140000E552E16ECCEF0EF0A4EC10F0BEEC0EF065
:1014100037EC10F00AE3D1EC10F0A90EEE58C30E31
:10142000EE58010EEE5801E2E7D0ADEC10F0A90E37
:10143000EE54C30EEE54010EEE540CE2BEEC0EF070
:10144000A00EEE5C2F0EEE58C50EEE58010EEE58B3
:1014500001E203D1BEEC0EF0F00EEE5C180EEE5879
:101460000D0EEE58030EEE580CE3E3EC10F0D00E28
:10147000EE54AC0EEE54110EEE54030EEE5401E396
:10148000BBD0BEEC0EF0500EEE5C380EEE581A0ECD
:10149000EE58030EEE580CE3E3EC10F0100EEE5491
:1014A000EF0EEE54200EEE54030EEE5401E3A4D0E2
:1014B000BEEC0EF0700EEE5C2C0EEE58290EEE58BF
:1014C000030EEE580CE3E3EC10F0500EEE54310E28
:1014D000EE54300EEE54030EEE5401E38DD0BEEC0C
:1014E0000EF0E00EEE5C0C0EEE58A60EB2EC0FF015
:1014F0000BE3BEEC0EF0600EEE5C270EEE58AC0E69
:10150000B2EC0FF001E2A9D01AEC11F0F00EEE5897
:10151000BC0EB2EC0FF004E3E6EC10F001E29DD05B
:10152000DFEC10F0320EEE58CC0EB2EC0FF009E307
:10153000D1EC10F04D0EEE58D20EB2EC0FF001E2ED
:101540008CD0DFEC10F0C80EEE58B30EB2EC0FF0FA
:1015500008E3D1EC10F0E30EEE58B90EB2EC0FF048
:101560004BE3E6EC10F008E31AEC11F0250EEE5810
:10157000C90EB2EC0FF040E3E3EC10F0600EEE5455
:10158000710EEE54580EEE540D0EEE5409E21AECA4
:1015900011F03A0EEE58690EEE580D0EEE585DE35E
:1015A000ADEC10F0DE0EEE54390EEE541A0EEE5481
:1015B00026E21AEC11F0290EEE58860EEE581A0E9D
:1015C000EE581DE2DBDB400EEE1808E1200EEE18AF
:1015D00005E1490EEE1802E11A0EEE1810E0CEDB1E
:1015E000600EEE1808E1C10EEE1805E1500EEE187F
:1015F00002E11A0EEE1803E0010EDF6E31D0E3ECCB
:1016000010F0400EEE54290EEE54860EEE541A0ED3
:10161000EE5425E2DFEC10F0740EEE58D20EEE58C8
:101620001A0EEE581CE2AADB800EEE1808E16B0ED3
:10163000EE1805E1950EEE1802E11A0EEE180FE015
:101640009DDBA00EEE1808E10C0EEE1805E19D0ED4
:10165000EE1802E11A0EEE1802E0DF6801D0DF6A30
:10166000DF50E55299D39CDB090EE12691EC10F096
:101670000ADEAEDB010E06C0DBFF020E07C0DBFF99
:10168000030E08C0DBFF040E09C0DBFF91EC10F075
:10169000BBDE69EC11F0DFCF14F0000EE76E14181A
:1016A000E8AE02D0143403D0E750D880145410E2CE
:1016B000010EDBCF14F0020EDBCF15F0030EDBCFF3
:1016C00016F0040EDBCF17F059DB8AEC0FF00AD0CE
:1016D000DFCF14F0143413E3CBEC0FF0D950010F2B
:1016E000E96EDCDB050E14C0DBFF060E15C0DBFF68
:1016F000070E16C0DBFF080E17C0DBFF0DD03EDB68
:10170000050EEECFDBFF060EEECFDBFF070EEECFB2
:10171000DBFF080EEECFDBFF050EDBCF14F0060E6D
:10172000DBCF15F0070EDBCF16F0080EDBCF17F07E
:10173000F2EC10F0090EE15C02E2E16AE552E16EC2
:101740002BD32EDB080EE12600018C5103E00101B2
:10175000050ED36F0101D351050A56E0010A3CE0A2
:10176000070A27E0010A16E0030A06E0010A01E081
:101770007BD040EC10F078D0FBEC10F0EE50010183
:10178000CB5D146EEE50CC59156EEE50CD59166EE1
:10179000EE501FD0FBEC10F00101CB51EE24146E83
:1017A000CC51EE20156ECD51EE20166ECE51EE20AE
:1017B00011D080C018F081C019F01A6A1B6A185045
:1017C000CB5D146E1950CC59156E1A50CD59166E4A
:1017D0001B50CE59176E0BD080C014F081C015F08D
:1017E000166A176ACB0EE96E010EEA6E93DB040EE1
:1017F00014C0DBFF050E15C0DBFF060E16C0DBFFB5
:10180000070E17C0DBFF30D08EDB2DDFE1DA040ED0
:1018100006C0DBFF050E07C0DBFF060E08C0DBFFBE
:10182000070E09C0DBFF49EC10F0EE500101CB19A7
:101830000CE1EE50CC1909E1EE50CD1906E1EE5065
:10184000CE1903E102E1D36B0FD049EC10F0EE505A
:10185000CB5DEE50CC59EE50CD59EE50CE5902E250
:10186000020E01D0010ED36F49EC10F09EDAC7DCF6
:10187000AFDA146E0F0E00018215141407E0010E8A
:101880008B6F40EC10F00101D36B0DD08B6B040E0D
:10189000DBCFCFF1050EDBCFD0F1060EDBCFD1F1E0
:1018A000070EDBCFD2F1080EE15C02E2E16AE552FD
:1018B000E16E72D275DA160EE1260001825102E164
:1018C000DF6A10D091EC10F09ADC82DAE76E010E3C
:1018D000E7CFDBFFDBCFE6FF000182390F0BE552DC
:1018E000E714DF6EDF5008E1010EDBCFE6FF0F0EDD
:1018F0008215E552E7148B6FDF5004E0030EDF6EB4
:101900000101D96FDF5001E0A1D0020EC7C1DBFF9A
:10191000030EC8C1DBFF040EC9C1DBFF050ECAC13F
:10192000DBFF060ECBC1DBFF070ECCC1DBFF080ED1
:10193000CDC1DBFF090ECEC1DBFF0A0ECFC1DBFF3D
:101940000B0ED0C1DBFF0C0ED1C1DBFF0D0ED2C1DF
:10195000DBFFFB0EDBCFC7F1FC0EDBCFC8F1FD0ECA
:10196000DBCFC9F1FE0EDBCFCAF129EC11F0C7C104
:1019700006F0C8C107F0C9C108F0CAC109F046ECB9
:1019800011F0FB0EDBCFCBF1FC0EDBCFCCF1FD0E6B
:10199000DBCFCDF1FE0EDBCFCEF1D3DE8CDB2CE046
:1019A000670A1FE0070A17E0020A06E0030A04E0DC
:1019B000020A24E16BDA24D0B4DBAEEC02F069EC6D
:1019C00011F0DF501DE100018C511AE1D3C1E6FF97
:1019D00013EC03F00ED0A5DBB1EC04F031EC11F008
:1019E00008D09FDB5CEC05F069EC11F0DF5008E1FA
:1019F00085DBE552DF6E04D0A3DA02D0DF68D96957
:101A0000DF5024E0020EDBCFC7F1030EDBCFC8F1BD
:101A1000040EDBCFC9F1050EDBCFCAF1060EDBCF1A
:101A2000CBF1070EDBCFCCF1080EDBCFCDF1090EE9
:101A3000DBCFCEF10A0EDBCFCFF10B0EDBCFD0F137
:101A40000C0EDBCFD1F10D0EDBCFD2F1DF50146ED7
:101A5000160EE15C02E2E16AE552E16E14509CD19F
:101A6000D9CFE6FF020E98D16FDB060EEFDA25E242
:101A7000FE0EDBCFD3F165DE1EDB1DE0670A17E04B
:101A8000070A10E0020A0AE0030A08E0020A03E07B
:101A9000DF68D96916D0050EDF6E12D09FDB13EC1C
:101AA00003F006D0D3C1E6FFF6EC04F001D026DB4C
:101AB000E552DF6E06D044DA04D0030EDF6E01017A
:101AC000D96FDF50E55268D13FDBFD0EDBCF80F0F0
:101AD000FE0EDBCF81F0EFDA1BE0670A12E0070AA7
:101AE0000CE0020A06E0030A04E0020A13E1CED980
:101AF00013D080D9E1EC02F007D07CD9F1EC04F0EE
:101B000003D078D992EC06F0E552E552DF6E04D0AE
:101B100017DA02D0DF68D969DF50E5523DD111DB19
:101B20000EE0030A0CE0010A0AE0070A08E0670A6F
:101B300004E0630A04E1AAD904D002DA02D0DF6823
:101B4000D969DF50E55228D1FCDA0EE0030A0CE037
:101B5000010A0AE0070A08E0670A04E0630A04E1F0
:101B600095D904D0EDD902D0DF68D969DF50E552AC
:101B700013D10101C6510BE0020ED96FCBC1DAF1CE
:101B8000CCC1DBF1CDC1DCF1CEC1DDF1000C050C27
:101B90000101C65108E0020ED96FD3C1DAF1DB6B47
:101BA000DC6BDD6B000C050CCCDA12E0030A10E0F4
:101BB000010A08E0600A04E0630A0AE167D90AD072
:101BC000BFD908D00BDBFBEC04F0E552DF6E02D08E
:101BD000DF68D969DF50E552DFD078DB11E0620AB7
:101BE0000BE0030A09E0010A04E0030A0CE14ED904
:101BF0000AD010EC05F002D0B8EC03F0DF6E03D091
:101C0000010ED96FDF6ADF50E552C6D05FDB11E00D
:101C1000620A0BE0030A09E0010A04E0030A0CE18E
:101C200035D90AD015EC05F002D0C1EC03F0DF6E17
:101C300003D0010ED96FDF6ADF50E552ADD081DAF3
:101C400012E0030A10E0010A08E0600A04E0630AF7
:101C50000AE11CD90AD074D908D0C0DA1AEC05F010
:101C6000E552DF6E02D0DF68D969DF50E55294D0CB
:101C700068DA0CE0030A0AE0010A1CE0600A04E0EA
:101C8000630A18E103D918D05BD916D0B3D82ADA81
:101C900003E183EC03F0DF6EDF5003E188EC03F037
:101CA000DF6EDF5003E100018B6B06D00001010EF7
:101CB0008B6F02D0DF68D969DF50E5526DD041DA11
:101CC0000CE0030A0AE0010A0FE0600A04E0630A7C
:101CD0000BE1DCD80BD034D909D08CD803DA06E17B
:101CE0007EEC03F0DF6E02D0DF68D969DF50E55289
:101CF00053D027DA0CE0030A0AE0010A0CE0600A7C
:101D000004E0630A08E1C2D808D01AD906D088ECEA
:101D100003F0DF6E02D0DF68D969DF50E5523CD0B6
:101D200010DA0CE0030A0AE0010A0CE0600A04E0A1
:101D3000630A08E1ABD808D003D906D079EC03F0E8
:101D4000DF6E02D0DF68D969DF50E55225D0F9D9BE
:101D50000CE0030A0AE0010A0CE0600A04E0630AEE
:101D600008E194D808D0ECD806D03BEC03F0DF6E45
:101D700002D0DF68D969DF50E5520ED0D950FB0F91
:101D8000D5EF10F0E66EE30EE66E010EE66EBBECEC
:101D900000F067DAD4EF01F0E552E7CFD9FF120087
:101DA000D9CFE6FFE1CFD9FF1200EECFE6FFEECFAD
:101DB000E6FFEECFE6FFEFCFE6FF1200E1C0E3F172
:101DC000E2C0E4F1E3C0E5F1E4C0E6F10101120094
:101DD00048DAE552120025DAC3D9F9EC34F005C02F
:101DE000EDFF04C0EDFF03C0EDFF02C0EFFFFC0EEE
:101DF000DB50C4D1FD0EDBCFE6FFEEEF10F0D95083
:101E0000F90FD3D9ADD958EC35F009C0EDFF08C0B2
:101E1000EDFF07C0EDFF06C0EFFF120006C0C7F1DF
:101E200007C0C8F108C0C9F109C0CAF129EF11F013
:101E30000D6A0E6AF2EF10F0E66EBCD918EC2CF0C9
:101E4000146E050E3EDA146E040EE15C12000E6A8A
:101E5000F9EC34F0010E02C0DBFF020E03C0DBFF21
:101E6000030E04C0DBFF040E05C0DBFF0101C651F9
:101E7000010A1200D950040FE66E000EDA20E66E59
:101E80001200E6520101C651010A1200050EDF6E72
:101E9000D96F1200DF50FE0BE84270D1DACFEAFFB3
:101EA000EE50185C146EEE501958156EEE501A581C
:101EB000166EEE501B58176E1200FD0EDBCF18F099
:101EC000FE0EDBCF19F0DF50040D1850F324E96E3D
:101ED0001950F420EA6E120006C0DEFF07C0DEFFD4
:101EE00008C0DEFF09C0DDFFDD52DD5211EF11F049
:101EF00002C014F003C015F004C016F005C017F0BE
:101F00001200CFC114F0D0C115F0D1C116F0D2C16A
:101F100017F01200EE501426EE501522EE50162245
:101F2000EE5017221200CBC1E6FFCCC1E6FFCDC1B7
:101F3000E6FFCEC1E6FF1200FCEC03F01EEF11F04D
:101F4000010ED96FDF6A12000F0B146E156A166A44
:101F5000176AE850DE261550DE221650DE22175092
:101F6000DD221200EE58080EEE581200F90EDBCFFB
:101F700014F0FA0EDBCF15F0FB0EDBCF16F0FC0EE3
:101F8000DBCF17F01200FB0EDBCF14F0FC0EDBCF23
:101F900015F03FEF11F0FB0EDBCF18F0FC0EDBCF9E
:101FA00019F0FD0EDBCF1AF0FE0EDBCF1BF0120096
:101FB000D950FC0FFAD8EE501200E66EF7EC07F09D
:101FC000166E0B0E4BEF11F000018D2715508E236E
:101FD00069D9EF6A000E12008F518F2BEA6A320F17
:101FE000E96E030EEA22FE0EDBCFEFFF1200DECF1A
:101FF00006F0DECF07F0DECF08F0DDCF09F0DD52CE
:10200000DD521200F9EC34F002C0C7F103C0C8F190
:1020100004C0C9F105C0CAF11200F86EF4CFF7FF91
:10202000F3CFF6FF040EF626000EF722F822120078
:10203000E552E552F3CF14F0F4CF15F01200FD0E87
:10204000DBCF14F0FE0EDBCF15F01200F36EFE0EA8
:10205000DBCFF4FFF350F45C1200156A8D25146E8B
:102060008E51152214C0E6FF15C0E6FF1200600E67
:10207000EE5C220EEE58C20EEE58010EEE58120023
:10208000CBC1CFF1CCC1D0F1CDC1D1F1CEC1D2F114
:102090001200D950040FE96EDACFEAFF1200D8809F
:1020A000000EEE5412008F51146E156A320E145C3D
:1020B000000E155812000101C651630A12009D88D6
:1020C0009D8A2EDEDF6EDF501200E80EE66E010EF6
:1020D000E66E47EF02F0160EE76FFD0EEA6F420E56
:1020E000E86F120040EC03F0E552E552DF6EDF507E
:1020F0001200FE0EDBCFE6FFE66A1200D3C1E6FF58
:1021000011EF06F0DF50146E050EE15C1200D9509D
:10211000010FE96EDACFEAFF48DE5AEC0CF069EF06
:1021200011F02CDED5EF0EF0E66E3C0EE66E020EE0
:10213000E66E5CEF11F0E76FFD0EE86F060EC2EF82
:102140000EF02EDE41EF0FF02BDEE6521200EDEC2A
:1021500000F0E552E552D4EF01F010DE4FEF10F041
:102160000A0E0B6E0C6A0D6A0E6AEECF06F0EECF09
:1021700007F0EECF08F0EFCF09F01200E76EFD0E8A
:10218000DBCFE9FFFE0EDBCFEAFFE750E926000ECA
:10219000EA221200E66EE66AE66A1EEC2AF0E8EF32
:1021A0000EF0ECDD000EEE5C1200E96EFF0EDA20A0
:1021B000EA6E1200D9CFE6FFDACFE6FF1200DEDDCD
:1021C000800EEE5C1200DADDD8801200D7DDC00E82
:1021D000EE5C0A0EEE58C30EB2EF0FF0FE0EDBCF30
:1021E000E6FF120014C006F015C007F016C008F094
:1021F00017C009F0120097DE43EC09F0E9DD6CEF3F
:102200000FF0FD0EE96F070EC2EF0EF0C9DD050EEF
:10221000E1261200C5DDDEEF0EF0C2DDFE0EDB5062
:102220001200D9CFE9FFDACFEAFF1200B9DD040EC0
:10223000E1261200A3DD400EEE5C12000101010E4A
:10224000D96F1200E66E16DE12EC34F0146E090E31
:102250001200800E0B6E960E0C6E980E0D6E0E6AAE
:102260001200E552E552E5521200C4DD31EC2CF0CB
:1022700018EF10F0DDDDF9EC34F078EF0FF0FD0E23
:10228000DBCF16F0FE0EDBCF17F0120058EC35F066
:10229000C5DD02EF10F0E15E1650146E156AFF0EF8
:1022A000161812008DC0E9FF8EC0EAFF1200E80E7A
:1022B0000B6E030E0C6E1200E66A8DEC07F069EFF0
:1022C00011F0E15E145076DFA7EF10F03DDF5BEF19
:0822D00010F07EDDDF6E12004C
:0822D800ABC2E6FFACC2E6FF59
:1022E000EDEC1BF0E552E552AAC2E6FFAEEC1BF0A6
:1022F000E552D9C21DFEB00EE66E020EE66EF5EC9A
:102300001BF0E552E552120058EC17F0E65292EC41
:102310001EF00F0E95120301FC6BFD6B8314DF6E34
:10232000FD0EE66E030EE66E640EE66E030EE66EBE
:10233000320EE66EFC0EE66E030EE66E960EE66E4E
:10234000030EE66EDFCFE6FF0BEC2EF0146E0A0EE6
:10235000E15E145078EC19F0CFEC29F09396939845
:102360009394270EE66EE66A040EE66E6B0EE66E3A
:10237000000EE66EB00EE66E020E86EC17F002015D
:10238000280EAB6F040EAC6FABC2E6FFE66E64ECDA
:102390001BF0E552E552F3CF64F2F4CF65F202018F
:1023A000180EAA6F140ED96F120EAF6F0E01010E28
:1023B0005B6F0201DA6B7F0EE66EE66AA3EC15F046
:1023C000E552E5527F0EE66E010E81EC17F07F0EAE
:1023D000E66E020E81EC17F0760EE66E030E81ECCF
:1023E00017F00201DB6BDC6BE5525DEF17F058EC88
:1023F00017F00301010EFD6FFE0EDBCF64F35DEFFE
:1024000017F058EC17F00301020EFD6FFD0EDBCF45
:1024100064F3FE0EDBCF65F35DEF17F058EC17F0B9
:102420000301050EFD6FFE0EDBCF64F3FA0EDBCF6A
:1024300065F3FB0EDBCF66F3FC0EDBCF67F3FD0E1F
:10244000DBCF68F35DEF17F058EC17F08EEC17F068
:1024500031EC2CF0E552E552F3CF14F0F4CF15F047
:10246000010EF3240301FD6F310EE66EE66A8EEC79
:1024700017F0640EE66E030EE66E64EC2CF0146E3C
:10248000060EE15E14505DEF17F058EC17F077EC94
:1024900017F03FEC2CF0E552E552E55207C014F07E
:1024A00008C015F009C016F0142A000E15221622D5
:1024B00014C0FDF3310EE66EE66A77EC17F0640E99
:1024C000E66E030E86EC17F05DEF17F0E6687F0E00
:1024D000E66EE66AE66AE66A61EC32F0050EE15EF7
:1024E000F3CFDBF2F4CFDCF21200DBC2E6FFDCC29A
:1024F000E6FF87DFE552E552120058EC17F0080EB0
:10250000E1260201DE5102E1010EDE6F0301FC5102
:1025100001E112D3030196513C0A01E1FED20C0AFB
:1025200001E165D1010A01E162D1030A01E15FD154
:10253000010A01E15CD1070A01E159D1010A01E177
:1025400056D1030A01E153D10E0A01E150D1010A2B
:1025500001E14DD1030A01E14AD1010A01E147D16C
:102560000C0A01E144D10A0A01E141D1030A01E167
:102570003ED1010A01E13BD17F0A01E138D1010AD4
:1025800001E135D1030A01E132D1010A01E12FD184
:10259000070A01E12CD1010A01E129D1030A01E175
:1025A00026D1010A01E123D10F0A01E120D1010A5C
:1025B00001E11DD1030A01E11AD1010A01E117D19C
:1025C000070A01E114D1010A01E111D1030A01E175
:1025D0000ED1680A01E106D1020A01E100D1070A21
:1025E00001E1F8D03E0A01E1F2D0010A01E1ECD0AC
:1025F000390A01E1E4D03E0A01E1D4D0010A01E147
:10260000C7D00A0A01E1BED01F0A01E1B7D0180AFB
:1026100001E1A8D0010A01E19ED0340A01E198D07D
:10262000370A01E192D0010A01E18CD0070A01E1E9
:1026300086D0010A01E180D0030A01E17AD0300A94
:1026400001E175D0010A71E03E0A66E0010A50E03E
:10265000120A48E0010A3EE0150A39E0120A32E0A7
:10266000010A2DE0030A24E00E0A17E0030A01E143
:10267000ABD0070A0FE0010A0AE01A0A05E0190ABE
:1026800001E05AD229DE58D269EC1CF055D270EC28
:102690001CF093D0D0EC1DF04FD23CEC1DF00009A3
:1026A00001E07ED006EC1EF0000901E183D078D075
:1026B000270E9CEC17F0B00EE66E020E59D097C3B1
:1026C000AAF23AD297C3ABF298C3ACF235D297C311
:1026D000D9F232D2F80EE66E6A0EE66E000EE66EA3
:1026E000D4DE53D098C3E6FF97C3E6FF2CDA4ED072
:1026F00097C3E6FF98C3E6FF64EC1BF0E552E55292
:10270000F3CF16FEF4CF17FE99C31CFE0E011189FC
:102710000201010EDA6F10D20201DA5101E10CD28E
:102720000E0111990201DA6B07D2D0DE05D2DDDE8F
:1027300003D297C36EFF00D297C36FFFFDD197C33B
:1027400070FFFAD197C371FFF7D197C372FFF4D12D
:1027500097C35BFEF1D1100E9CEC17F0940EE66E61
:10276000020E06D0040E9CEC17F0A50EE66E020ECB
:10277000E66E64EC2CF0146E060EDCD163DB81ECAB
:1027800019F003D05FDBDAEC19F0E552E5521AD00C
:102790003CEC1DF0000904E106EC1EF000090AE023
:1027A000010E0BD046EC1DF0000906E10CEC1EF00A
:1027B000000902E1000E01D0010EE66E02D073CFD7
:1027C000E6FF15DEE552B8D11DEC1DF0B5D135ECB4
:1027D0001DF0B2D1958E959C0301FA81ADD1030114
:1027E000FA83AAD197C3FBF396908490A5D1030EE8
:1027F00097C3DBFF040E98C3DBFF050E99C3DBFF15
:10280000060E9AC3DBFF010EF36E070EF3CFDBFF5C
:1028100096514E0A01E161D1030A01E15BD1010A3F
:1028200001E155D1070A01E14FD1010A01E13ED191
:10283000030A01E133D1010A01E112D10F0A01E1DA
:1028400005D1010A01E1FFD0030A01E1F9D0010A33
:1028500001E1ECD0070A01E1D1D0010A01E1C4D0C5
:10286000030A01E1BDD0010A01E1B1D07F0A01E113
:10287000A5D0010A01E195D0030A01E185D00A0A39
:1028800001E17FD00C0A01E179D0010A01E173D0A6
:10289000030A62E0010A59E00E0A51E0030A48E027
:1028A000010A42E0070A31E0010A28E0030A1FE0BA
:1028B000010A01E018D15ADB01E215D1030EDBCF8A
:1028C000DDF2DDC2E6FF0FEC07F0E552E76E070E22
:1028D000E7CFDBFFDB5002E00201DD6BDDC2E6FF8C
:1028E000050EE66EA6EC1EF0E552E552FCD03EDB8E
:1028F00001E2F9D041DB37EC07F0DED024DB01E365
:10290000F2D0C1DA5FEC07F0D6D096DA800EEE5C3A
:10291000960EEE58980EEE58000EEE5801E3E3D0F6
:1029200028DB8DEC07F00ED024DB5AEC0CF00AD03B
:102930000ADB01E3D8D0A7DABCEC07F0BCD019DB86
:1029400030EC0DF0E552E552B6D010DB01E2CBD011
:1029500013DB34EC0DF0B0D06FDA000EEE5C000E3D
:10296000EE58010EEE58000EEE5801E3BCD08BDAA3
:1029700064EC0DF0A0D08FEC0DF0B1D0A4EC0DF014
:10298000AED0B9EC0DF0ABD0030EDBCF83F0040E6C
:10299000DBCF84F0050EDBCF85F0060EDBCF86F0B3
:1029A00043D0030EDBCF87F0040EDBCF88F0050E9B
:1029B000DBCF89F0060EDBCF8AF036D083C0DAF1A8
:1029C00084C0DBF185C0DCF186C0DDF113D087C0A7
:1029D000DAF188C0DBF189C0DCF18AC0DDF10AD010
:1029E000030EDBCF82F020D082C0DAF10101DB6B75
:1029F000DC6BDD6B0101020ED96F4DD0030EDBCF16
:102A000014F0040EDBCF15F0050EDBCF16F0060E2A
:102A1000DBCF17F0145015101610171002E1000E3E
:102A200001D0010E00018C6F010E49D005DA210E94
:102A3000EE5C000E2DDA38E29FDAD4EC0DF03CD0DB
:102A4000EDEC0DF04CD006EC0EF049D0F5D9000EAF
:102A5000EE5C010E1DDA28E28FDA1FEC0EF02CD0AE
:102A6000010E63DA04E00001010EE56F02D00001FF
:102A7000E56B020E5ADA04E00001010EE66F02D0A7
:102A80000001E66B040E51DA04E00001010EE76F6D
:102A900002D00001E76B070EDB6A25D05ADA04E2A8
:102AA000F2D938EC0EF007D0030E09D052DA06E264
:102AB000EAD95FEC0EF0E552E55211D0030EF36E49
:102AC000070EF3CFDBFF0FD079EC0EF008D090ECBF
:102AD0000EF005D0A7EC0EF002D0C8EC0DF0E76EBA
:102AE000070EE7CFDBFF070EDB5004E0070EDBCF5E
:102AF000DEF209D00101D95103E0D9C1DEF203D0E1
:102B00000201010EDE6F0201DE0516E100018B51AC
:102B100013E00201020EDE6F0FD0DAC1E6FFDBC167
:102B2000E6FFDCC1E6FFDDC1E6FFDEC2E6FF76DCE4
:102B3000146E050EE15E1450080EE15C02E2E16ADB
:102B4000E552E16EBAD1B4D9020EE12681948198A2
:102B5000FE0EDB50020B020802E0000E01D0010E57
:102B6000E8B08186E8A0819681888198FE0EDB50CE
:102B7000010BE8B08186E8A0819681888198DE52B9
:102B8000800EDD6E080EDF6EDF501EE0010EDBCF23
:102B9000E6FFFD0EDB50E552E714146E010EDB502C
:102BA000145C02E0000E01D0010EE8B08186E8A0BE
:102BB000819681888198010EDBCFF3FFF390F34279
:102BC000F3CFDBFFDF06E0D78184020EE15C02E297
:102BD000E16AE552E16E71D10301FAA113D1030E4E
:102BE0000101C65D01E094D00301FE51030A6CE0CF
:102BF000010A50E0030A2AE0010A06E0FE6B020E19
:102C0000FA1501E182D07ED0020EFA1504E06BD9EC
:102C100006E0010E04D08350800B01E0010E000994
:102C20000EE0010EFE6F0E01140E5C6FCFC1E6FFC9
:102C3000D0C1E6FFD1C1E6FFD2C1E6FF90D1020EBE
:102C4000FA1502E0838C010C839C000C020EFA152D
:102C500004E049D906E0010E04D08350800B01E066
:102C6000010E00090AE1FE6B020EFA1503E0838CE7
:102C7000010E02D0839C000E24D10E015C5101E0B4
:102C8000DAD00301020EFE6FFA1502E0839C000CFD
:102C9000838C010C020EFA1504E025D906E0010E22
:102CA00004D08350800B01E0010E000901E0C3D085
:102CB000030EFE6F020EFA1502E0838C01D0839C96
:102CC0000E01010E5C6F1200020EFA1504E00BD922
:102CD00006E0010E04D08350800B01E0010E0009D4
:102CE00008E0020EFE6FFA1502E0839C000C838C54
:102CF000010C0E015C5101E09ED00301FE6B020E3F
:102D0000FA1503E0838C010E02D0839C000ED9D00B
:102D10000301FB5160E0FE51030A3AE0010A25E09D
:102D2000020A05E0FE6B020EFA1565E052D0020EB3
:102D3000FA1504E0D8D806E0010E04D08350800BC9
:102D400001E0010E000909E0020EFE6F8490FA1501
:102D500002E0839C000C838C010C020EFA1502E049
:102D6000838C01D0839C84901200020EFA1504E03B
:102D7000BAD806E0010E04D08350800B01E0010EAA
:102D8000000959E1030EFE6F8480FBC35CFE120054
:102D9000020EFA1504E0A7D806E0010E04D0835015
:102DA000800B01E0010E000907E0020EFE6F849027
:102DB000FA150BE0839C000C0E015C513CE1030111
:102DC000FE6B8490020EFA1502E0838C010C839C4A
:102DD000000C838C010C020EFA1504E084D806E086
:102DE000010E04D08350800B01E0010E000905E0C4
:102DF000020EFA1505E0839C000C020EFA1512E093
:102E0000838C010C020EFA1504E06DD806E0010E69
:102E100004D08350800B01E0010E000905E0020E92
:102E2000FA1505E0839C000C020EFA1502E0838C73
:102E3000010C839C000E1200D950030FE96EDACF0B
:102E4000EAFF1200030E78D8D9CFE6FFDACFE6FF0B
:102E500080EC2BF0146E060EE15E1450020EDBCFF8
:102E6000E6FFDECFE6FFDDCFE6FF1200EE501416E0
:102E7000EE501516EE501616EE501716145015108B
:102E800016101710120078D8040EDBCFE6FF1200E0
:102E9000EE58000EEE58000EEE581200D880FF0ECD
:102EA000EE54000EEE54000EEE54000EEE541200DE
:102EB000D9CFE6FFE1CFD9FF1200E552E7CFD9FF26
:102EC0001200CBC1E6FFCCC1E6FFCDC1E6FFCEC10B
:102ED000E6FF45D0EECFE6FFEECFE6FFEECFE6FF12
:102EE000EFCFE6FF12008350800B800A1200FC0E29
:102EF000DBCFE6FFFD0EDBCFE6FFFE0EDBCFE6FF0E
:102F00001200E66E20DEE552E5521200E66E92EC0B
:102F10002CF0146E070EE15E14501200FD0EDBCF94
:102F2000E6FFFE0EDBCFE6FF1200146E156A166A8E
:102F3000176A82DF36EF17F0E66EE66A970EE66EE6
:102F4000030EE66E120078DF100EEE5C270E48EFDF
:102F500017F072DFFF0EEE5CFF0E48EF17F0B1ECDA
:102F600004F0E552E552E552E552120065DF4EEFFE
:102F700017F062DF6AEF17F0030EDBCFE6FF1200F7
:102F8000000306090C101316191C1F2225282B2ECE
:102F9000313336393C3F414447494C4E51535558E3
:102FA0005A5C5E60626466686A6B6D6F70717374A0
:102FB000757678797A7A7B7C7D7D7E7E7E7F7F7F59
:102FC0007F7F7F7F7E7E7E7D7D7C7B7A7A7978763F
:102FD00075747371706F6D6B6A68666462605E5C55
:102FE0005A585553514E4C494744413F3C3936336A
:102FF000312E2B2825221F1C191613100C0906032D
:1030000000000000000000000000000000000000C0
:1030100000000000000000000000000000000000B0
:1030200000000000000000000000000000000000A0
:103030000000000000000000000000000000000090
:103040000000000000000000000000000000000080
:103050000000000000000000000000000000000070
:103060000000000000000000000000000000000060
:103070000000000000000000000000000000000050
:103080000000000000000000000000000000000040
:103090000000000000000000000000000000000030
:1030A0000000000000000000000000000000000020
:1030B0000000000000000000000000000000000010
:1030C0000000000000000000000000000000000000
:1030D00000000000000000000000000000000000F0
:1030E00000000000000000000000000000000000E0
:1030F00000000000000000000000000000000000D0
:1031000000000000000000000000000000000000BF
:1031100000000000000000000000000000000000AF
:10312000000000000000000000000000000000009F
:10313000000000000000000000000000000000008F
:10314000000000000000000000000000000000007F
:10315000000000000000000000000000000000006F
:10316000000000000000000000000000000000005F
:10317000000000000000000000000000000000004F
:10318000D8EC20F01468156AFD0EDBCF08F0FE0EB7
:10319000DBCF09F014C00DF015C00EF0B3EC35F024
:1031A00008C0DEFF09C0DDFF0EEC20F0EE50ED1090
:1031B00009E0E66A9CEC35F0E552DF06010EF4E228
:1031C000DB06F2D7CEEC1FF00D680E6A14C008F0D3
:1031D00015C009F0B3EC35F004C014F005C015F0CB
:1031E00004C0DEFF05C0DDFF0EEC20F0EE50ED1058
:1031F00005E0DFCFE6FF9CEC35F0E552020EE15C26
:1032000002E2E16AE552E16EE8EF1EF0010ED16ED6
:103210001200D16A12000201635101E104001200A0
:103220000201010E636F1200ADEC20F07EEC20F085
:10323000FB0EDBCFEEFFFC0EDBCFEDFFDF5001E03E
:103240009D80E552E8EF1EF0E3EC1EF0030EE12650
:10325000E5EC20F0EDCFDBFFDF5001E09D803CECA2
:1032600020F04AEC20F0030EE15C02E2E16AE55254
:10327000E16EE8EF1EF0ADEC20F07EEC20F0F90EF0
:10328000DBCFEEFFFA0EDBCFEEFFFB0EDBCFEEFF68
:10329000FC0EDBCFEEFFDF5001E09D80E552E8EF52
:1032A0001EF0DCEC20F0E5EC20F0EECFDBFF030EAF
:1032B000EECFDBFF040EEECFDBFFDF5001E09D80A1
:1032C0003CEC20F0030EDBCF16F0040EDBCF17F042
:1032D00014C006F015C007F016C008F017C009F0BA
:1032E000050EE15C02E2E16AE552E16EE8EF1EF0F4
:1032F0000201936B93C292F293C27CF293C27BF26F
:103300001200ADEC20F002017B29DF6E070EDF5CBE
:1033100001E3DF6A7C51DF5C02E1010E2ED07B51BC
:103320006EEC1FF043EC20F07B516EEC1FF02EECA6
:1033300020F0DFCF7BF2CEEC1FF0000E1416F00E63
:103340001516145002E1200E15180FE0FD0EDBCF0C
:1033500016F0FE0EDBCF17F0000E1616F00E171645
:1033600016500AE1100E171807E1FD0EDB50010B95
:1033700003E10F01010E736F000EE552E8EF1EF03E
:10338000E3EC1EF002017C517B5D02E1010E10D0E6
:103390007C516EEC1FF0B0EC20F07C516EEC1FF015
:1033A000BBEC1FF07C2B070E7C5D01E37C6B000EF9
:1033B000E8EF1EF0ADEC20F002019229DF6E070E5F
:1033C000DF5C01E3DF6A9351DF5C02E1010E0DD0A7
:1033D000925178EC1FF043EC20F0925178EC1FF002
:1033E0002EEC20F0DFCF92F2000EE552E8EF1EF057
:1033F000E3EC1EF002019351925D02E1010E10D048
:10340000935178EC1FF0B0EC20F0935178EC1FF062
:10341000BBEC1FF0932B070E935D01E3936B000E43
:10342000E8EF1EF0DCEC20F027DB000970E1F1ECA6
:103430001FF0A6DFA5EC20F0000969E11FEC20F0E9
:1034400006E2F3EC1EF0A7DAA5EC20F060D0010E46
:10345000DB50C00B2BE059EC1FF0DBCF01F2040E68
:10346000DBCF02F2010EDB50800B0DE037EC1FF0DA
:10347000F5CF00F20201046B056B72CF03F2076B0C
:10348000086B066B07D00201C80E006F010E046FB7
:10349000056B036B020EDBCF1AFEDBCF57FE2CEC65
:1034A0001FF09D900E0136899D8031D018EC20F0E0
:1034B00015E1100E151812E1020EDBCFE6FF71CFF9
:1034C000E6FF70CFE6FFBEEC20F0D890E936EA3692
:1034D000E806FBE1A1EC1FF01AE117D018EC20F090
:1034E00016E1200E151813E1020EDBCFE6FF6FCFB9
:1034F000E6FF6ECFE6FFBEEC20F0D890E936EA3664
:10350000E806FBE1A1EC1FF002E10F01736B050E71
:10351000E15C02E2E16AE552E16EE8EF1EF0DCEC0C
:1035200020F0B4DA000932E1F1EC1FF061DFA5EC24
:1035300020F000092BE11FEC20F006E2F3EC1EF076
:103540005BDAA5EC20F022D0010EDB50800B1EE0F0
:1035500059EC1FF0DBCF01F1040EDBCF02F137ECA9
:103560001FF0F5CF00F10101046B056B72CF03F181
:10357000076B086B066B020EDBCF1CFEDBCF59FE20
:103580002CEC1FF09D900E01368D9D80050EE15CA8
:1035900002E2E16AE552E16EE8EF1EF0E3EC1EF0B4
:1035A000FE0EDB50200A01E17FD0290A01E17CD028
:1035B000530A70E00E0A64E0770A5AE0670A50E0A6
:1035C000070A4BE0010A46E0030A41E06B0A37E0D4
:1035D0001A0A2DE0090A28E0010A23E00F0A1EE07A
:1035E000010A19E0030A14E0010A0FE0070A0AE0E1
:1035F000010A05E0030A60E1AAEC20F022D0AAEC5F
:1036000020F017D0AAEC20F035D090EC20F019D0A3
:1036100090EC20F00ED090EC20F02CD095EC20F027
:1036200010D095EC20F005D095EC20F023D09AEC4A
:1036300020F04CEC1FF0060EEE6E230E43D09AECF9
:1036400020F04CEC1FF0B10EEE6E1F0E3BD0AAEC3A
:1036500020F008D090EC20F005D095EC20F002D0BE
:103660009AEC20F04CEC1FF0CF0EEE6E2A0E2AD012
:103670009AEC20F04CEC1FF0B80EEE6E260E22D025
:103680009BDB2D0EEE6E090E4CEC1FF0890EEE6EDC
:103690000B0E18D091DB950EEE6E0C0E4CEC1FF05D
:1036A000410EEE6E100E0ED087DBEE6AED6ACBECAB
:1036B00020F0EE6AED6A07D0AAEC20F0EDDB450EB3
:1036C000EE6E120EED6E84D37EDB040EE126CEECA0
:1036D0001FF014C0DFFF010E15C0DBFF020EDB6A16
:1036E000030EDB6A0EEC20F0FD0E0B6EB50E0C6EB9
:1036F000060E0D6E0E6AEECF06F0EECF07F0EECF9F
:1037000008F0EFCF09F0F9EC34F005C0EDFF04C08C
:10371000EDFF03C0EDFF02C0EFFF0EEC20F0EE5214
:10372000800EEE26000EEE22EE220EEC20F04FEC84
:1037300020F0EECF16F0EFCF17F0100ED890173222
:10374000163215321432E806F9E14AEC20F0040E84
:10375000E15C02E2E16AE552E16E3AD3ADEC20F0C1
:10376000050EF36EFE0EDBCFF4FFF350F45C05E2C2
:10377000050EF36EFE0EF3CFDBFFFE0EDB50166E72
:10378000176AFE0EDB5025EC20F014C008F015C0BF
:1037900009F016C00DF017C00EF0B3EC35F008506C
:1037A000DF6EDFCF37FE0E013751E8240E01386F90
:1037B000030E0E013703F3CF39FE040E3703F3CFA8
:1037C0003AFEDF5025EC20F014C009F0DFCF0EF0F8
:1037D000E7EC35F00950E552FBD2F5DA9FEC20F02A
:1037E000F3CF64F2F4CF65F2F3D2EDDA040EE12602
:1037F0009D900E0136919D800E01C80E446F030E00
:10380000456F020E44CEDBFF030E45CEDBFFDF6AC1
:10381000DF6ADF5084EC20F0EF503CE0310EDF5CDB
:1038200039E2DF5084EC20F0EF507F0BE76E010EA1
:10383000E7CFDBFFDBCF14F05F0EE76E1418E8AEC6
:1038400002D0143403D0E750D88014540AE2200E7A
:10385000146E010EDBCFE7FF1450E75E010EE7CFD9
:10386000DBFF280E146E4E0E156E000E166E010E46
:10387000DBCF17F0186A196A17AE02D018681968FA
:103880006FEC20F0F550E66E90DBE552E750EF6EFE
:10389000DF2ABFD78ADBEF6A0E01466B64C218FECF
:1038A00065C219FE9D903F0E0E0111170E01368163
:1038B0009D80040EE15C02E2E16AE552E16E88D28D
:1038C000B7EC20F085D2B7EC20F00E0136B1FDD771
:1038D0007FD29D900E0136910E01119D9D801200A8
:1038E000400E0E011115146E010E0E013615141046
:1038F0001200ADEC20F0DF6AD2DA0800F55010E0DB
:10390000F90EDB50DF5C0CE2D3DBD950FD0FACDBF2
:10391000EF22D950FA0FA8DBEE22EE22DF2AECD7F5
:10392000C7DBE55255D24FDAFE0EDB50040A32E017
:10393000070A1CE0010A0EE0030A2CE19D900E012B
:1039400036990E011191DEDA000EE66E020E38DBBA
:1039500083DA20D09D900E01369B0E011195D2DAAC
:10396000630EE66E010E2CDBE1DA14D09D900E01A1
:10397000369D0E011199C6DA000EE66E010E20DBAF
:103980000E01000E4B6F010E4C6F0E01000E536FB7
:10399000010E546F1DD2E1DBDF6A4FD853DA37DBFB
:1039A00009E050DADEDA010EF4DADBCF1AFEDBCF03
:1039B00057FEDF88AEDB2BDB18E0ABDB0900F550F0
:1039C0000900F5CFE7FF0800F5CFF8FFE7CFF7FFD5
:1039D000F66E0800F55009E09CDBC3DA020ED9DA76
:1039E000DBCF1BFEDBCF58FEDF8A9D90DF500E0140
:1039F00036139D80E552ECD1E6D937D823DA07DBC0
:103A00000CE020DAAEDA030EC4DADBCF1CFEDBCF2B
:103A100059FE9D900E01368D9D80DAD1D4D90DD8F6
:103A20008EDBF3CF12FEF4CF13FEFC0EDBCF1AFEBB
:103A30009D900E0111819D80CBD19D90CF0E0E01E6
:103A40003617FA0E0E0111179D801200BCD90DD841
:103A500076DBF3CF16FEF4CF17FEFC0EDBCF1CFE99
:103A60009D900E0111899D80B3D19D900E01369DD0
:103A70000E0111999D801200300E0E01361505E1E0
:103A8000050E0E01111501E1000C010C400E0E0196
:103A9000361505E1100E0E01111501E1000C010CA7
:103AA0005CDBCBDF3CDA31EC2CF0E552E552110E59
:103AB000F35C000EF45803E3100E26DBEF6A0E01F0
:103AC000000E476F020E486F0E01630E496F010E24
:103AD0004A6FFD0EDBCFE9FFDB2AFE0EDBCFEAFFEC
:103AE00001E3DB2AEFCFDFFFDF5028E070DAFC0EC6
:103AF00059DB72DAEE52E9CF14F0EACF15F0E9CFD4
:103B0000E6FFEACFE6FF63DAEE52E9CF16F0EACF3E
:103B100017F0E9CFE6FFEACFE6FFDFCFE6FF3EDDB5
:103B2000186E050EE15E185067DA51DAFB0E3ADBCB
:103B30002CDBEE52EE6AED6A5FDACBD748DAEF6A39
:103B400024DBEF6A49DAEE52EE6AED6A85D9EED9E6
:103B5000FA0EDBCF1BFE1BCE1AFEDBCF58FE58CE73
:103B600057FE9D90300E0E0136139D80E55230D1E8
:103B70002AD963DF140EE66E0E0EE66E120EE66EA6
:103B80000E0EE66EFE0EDBCFE6FF08DD146E050EB0
:103B9000E15E14509D90050E0E0111139D8018D109
:103BA0004CDF0201640E006F0101636F0201950E8C
:103BB000016F0C0E026F0101410E646F100E656FF4
:103BC0000201640E036F0101666F0201046B056B55
:103BD0000101676B686B0201066B0101696B010EE5
:103BE0000201076F086B01016A6F6B6B35D99ED9B3
:103BF0009D90300E0E0136139D801200300E0E0186
:103C000036151200400E0E013615120002017C51CD
:103C10007B5D01E1000C010C02019351925D01E119
:103C2000000C010C9ADAFE0EDBCFE6FFE66A31ECFF
:103C300035F0E552E552F350F41004E0FE0EDB508F
:103C4000D00F04D0FE0EDB50BF0F0A0FDF6EDF5027
:103C5000E552BED0ADDAFD0EDBCFDEFFDBCFDDFF00
:103C6000E2D9EF5005E0DF2A010EFAE3DB2AF8D7AC
:103C7000DAD9FC0EDBCFEFFFD6D9010EACDAEF6A52
:103C80008DD908DA020EE15C02E2E16AE552E16EEA
:103C90009FD09D929F82D08EF90E94160F0EBD6E0E
:103CA000BA6E1C0ECA6ECB680E01116B0E017F0E30
:103CB0001E6F0E011A6F0E011B6F0E011C6F0E019D
:103CC0001D6F0E01370E126F1A0E136F0E01370E95
:103CD000146F1A0E156F0E01370E166F1A0E176F2E
:103CE0000E01370E186F1A0E196F1200810ECD6E6D
:103CF0009F90140EE66E32DDE552E80EE66E030E7E
:103D0000E66E6BDDE552E5520E017F0E5A6F5ACE1C
:103D100059FE5ACE58FE5ACE57FE0E01366B0E0192
:103D20003B6B1200870ED56EB16AF18EF26A9D6A06
:103D3000A06AAFDF76EF1EF046D8AA6AFE0EDB500F
:103D4000A96EA69EA69CA680A85042D031DAA19862
:103D5000AA6AFE0EDB50A96EFD0EDB50A86EA69E71
:103D6000A69CA684F250800B01E0010EDF6EF2509B
:103D7000400B01E0010EE76E010EE7CFDBFFF29E84
:103D8000F29C550EA76EAA0EA76EA682DF50E8B071
:103D9000F28EE8A0F29E010EDB50E8B0F28CE8A0B3
:103DA000F29CA1A8FED7A198A694020EE15C02E2C3
:103DB000E16AE552E16E0CD0FC0EDBCFE9FFFD0EAF
:103DC000DBCFEAFF1200D9CFE6FFE1CFD9FF120027
:103DD000E552E7CFD9FF1200FD0EDBCFE9FFFE0E63
:103DE000DBCFEAFF1200020EDBCFE6FF3F0E176EBD
:103DF000520E186E000E196EDECF1AF0DDCF1BF0DA
:103E00001C6A060E0C6E0D6A0E6A1AC007F01BC003
:103E100008F01CC009F09CEC33F004C01AF005C097
:103E20001BF006C01CF017500424146E1850052017
:103E3000156E19500620166E14C0E6FF15C0E6FF79
:103E4000E66E1200FC0EDBCFF6FFFD0EDBCFF7FFB8
:103E5000FE0EDBCFF8FF12000E01000E476F020EC0
:103E6000486F0E01000E4F6F020E506F1200950E3C
:103E7000146E530E156E000E166EDECF17F0DDCFEA
:103E800018F01838186A0F0B176E070E1716000E69
:103E90001816196A6FEF20F0ED6ECBEF20F0FA0ED6
:103EA000DBCFF6FFFB0EDBCFF7FFFC0EDBCFF8FF1F
:103EB000120086D9FF0E14160F0E151614C0E6FF59
:103EC00015C0E6FF64EC1BF0E552E552030EF3CF9C
:103ED000DBFF040EF4CFDBFF030E1200030DF3CF64
:103EE000E9FFF4CFEAFF660EE926020EEA2212008D
:103EF000030DF3CFE9FFF4CFEAFF7D0EE926020EB2
:103F0000EA2212009D80210EE66EFB0EDBCFE6FF5B
:103F1000FC0EDBCFE6FFFD0EDBCFE6FF1200FD0E51
:103F2000DBCFE6FFFE0EDBCFE6FF12000E01630ED5
:103F3000496F010E4A6F0E01630E516F010E526FF1
:103F40001200740EE9260F0EEA22EECFE6FFEFCF45
:103F5000E6FFA6DD146E050EE15E1450DF50010B86
:103F600012000900F5CFE6FF0900F5CFE6FF0800D3
:103F7000F5CFE6FF1200020E2ED9EF50E66EFB0ED3
:103F8000DBCFE9FFFC0EDBCFEAFFE552E750EF6E37
:103F90001200E66EC8DCD9D8FB0E1200FD0EDBCF96
:103FA00014F0FE0EDBCF15F01200DF50E76E020EAC
:103FB000DBCFE9FF030EDBCFEAFFE750EBEF20F0AA
:103FC000E66E97DC146E060EE15E1450120047CECA
:103FD000E9FF48CEEAFF120049CEE9FF4ACEEAFFE8
:103FE0001200D950020FE66E000EDA20E66ED9CF2D
:103FF000E6FFDACFE6FF12000E01030E4727000EA0
:1040000048230E01030E4927000E4A23120009001F
:10401000F5500900F5100800F5101200D9CFE9FF9E
:10402000DACFEAFF1200DECFE9FFDDCFEAFF1200B0
:10403000C7D8000E1416F00E151614501200C0D872
:10404000390E145C000E15581200156AE8307F0B0B
:10405000146EF00E1426000E15221200020EBBD8AC
:10406000FC0EDBCFEFFF1200E96EFF0EDA20EA6EE6
:10407000030EEE26000E1200010EDBCF14F0020E2E
:10408000DBCF15F01200FD0EDBCFEEFFFE0EDBCF17
:10409000EDFF120014C0F3FF15C0F4FF1200EECFC5
:1040A00014F0EECF15F01200450EEE6E120E120057
:1040B000F6DE0800F550E66E8FDEE552E750EF6E53
:1040C000EEDE09000900F5CF15F00800F5CF16F077
:1040D00083DEEE5215C0EEFF16C0EDFF1200145045
:1040E0001724F36E15501820F46E16501920F86E30
:1040F000F4CFF7FFF3CFF6FF080012009D50010B3D
:10410000DF6E9D90ECEF1EF0E76E66DEE750EBEFA2
:1041100020F098DE030EF626000EF722F822120099
:104120004BDE2F0EEE6E140E120046DE560EEE6EB5
:10413000160E120041DEAB0EEE6E180E1200EFDE10
:1041400064EC1BF0E552E5521200E552E552E552EF
:10415000E552120031DE54EF20F035DEE652120057
:104160009EDF3ADE14C0EEFF15C0EDFF12002BDE1D
:10417000D6DEF5EC1BF0E552E552120054DF010EDD
:10418000E916000EEA16010E120021DFEE52EE6A69
:10419000ED6AECEF1FF0FA0EDBCFE9FFFB0EDBCF91
:1041A000EAFF1200DBCFEFFF17DFDBCFEFFF1200DC
:1041B0000ADE020EE126120006DE050EE1261200DE
:1041C000DECF14F0DDCF15F0120098DF010EEECF38
:0E41D000DBFF020E1200E926000EEA221200AA
:0241DE002BECC8
:1041E00026F0FB0EDBCFF3FFDB06F35000090AE0FD
:1041F00079EC26F0FA0EE4EC26F0F3E1151CF1E17F
:10420000010E01D0000E5AEF26F02BEC26F03B0EEB
:10421000E12402E3E168E652E16E010EDB6A020E80
:10422000DB6AF90EDBCFF6FFFA0EDBCFF7FFFB0EF2
:10423000DBCFF8FF0800F550DF6EDF5002E17EEFC4
:1042400025F0250EDF5C02E071EF25F0030EDB6A3E
:10425000040EDB6A050EDB6A060EDB6A070EDB6AFC
:1042600093EC25F02D0EDF5C0CE02B0EDF5C09E0FB
:10427000200EDF5C06E0230EDF5C03E0300EDF5C27
:104280001AE1DF50300A14E0130A0FE0030A0AE0D3
:104290000B0A05E0060AE4E1030EDB80E1D7030E1A
:1042A000DB82DED7030EDB84DBD7030EDB86D8D7B9
:1042B000030EDB88D5D72A0EDF5C1BE18FEC25F0DF
:1042C000DDEC25F010E0030EDB8008680968130EB2
:1042D000DBCF0DF0140EDBCF0EF0E5EC33F0040E67
:1042E00006C0DBFF03D0130EC6EC25F093EC25F0DF
:1042F0000BD0090EDB6A34EC26F003E0A8EC26F0C4
:10430000FAD7090EC6EC25F0030EDBB0DB982E0EB3
:10431000DF5C1BE193EC25F02A0EDF5C0BE18FECF8
:1043200025F0DDEC25F003E1130E18EC26F093ECFC
:1043300025F00BD0090EDB6A34EC26F003E0A8EC84
:1043400026F0FAD7090E18EC26F0680EDF5C07E1BC
:1043500093EC25F0680EDF5C1DE1030E18D0740E9F
:10436000DF5C17E07A0EDF5C14E0480EDF5C06E0ED
:10437000540EDF5C03E05A0EDF5C02E1020E07D050
:104380006C0EDF5C03E06A0EDF5C04E1010E6BEC97
:1043900026F0C9DBDF506E0A01E17FD31E0A01E17E
:1043A00092D1200A01E18FD13F0A01E149D11A0AD5
:1043B00001E146D10D0A01E143D1200A01E140D1DA
:1043C0003A0A01E13DD1200A01E13AD1260A01E190
:1043D00035D10D0A01E132D11A0A01E1D9D0200A02
:1043E0004AE0300A1FE0460A0EE0250A01E083D3C6
:1043F000D950F90FE96EFF0EDA20EA6E010EEE5E7B
:10440000000EEE5AEE5A79EC26F0250EE66E95DB9C
:1044100003E1151C01E169D375EC26F001E26BD3D1
:10442000DB2A69D3080EDB6A040EDB50010806E2C2
:10443000040EDB043DEC26F0DB508BDB080EDB507A
:1044400009E0030EDB50010B05E172DB01E04DD307
:10445000080EDB6A64DBEFCFDFFFEDEC26F003E153
:10446000151C01E142D375EC26F001E3DB2A60DB89
:1044700001E141D33AD3070EDB5002080FE1B9EC5A
:1044800026F0030E80EC26F00E0EEECFDBFF0F0EB3
:10449000EECFDBFF100EEECFDBFF20D0F70EDBCF31
:1044A00017F0F80EDBCF18F0020E175E000E185A48
:1044B000F70E17C0DBFFF80E18C0DBFF17C0E9FFCF
:1044C00018C0EAFF70EC26F0166A0E0E14C0DBFF6F
:1044D0000F0E15C0DBFF100E16C0DBFF0E0EDBCF7C
:1044E000E6FF0F0EDBCFE6FF100EDBCFE6FF3FEC63
:1044F0002CF0E552E552E552130E07C0DBFF140E17
:1045000008C0DBFF060EDB5005E0130EB4EC26F00E
:1045100001E26ADBD8EC26F002E2130E37DB9BECFB
:1045200026F006E0040EB4EC26F002E2050E2EDBC7
:10453000030EDBB005D0FCDA01E0D7D2080EDB6A4F
:10454000090EDB6A0E0EDBCFF6FF0F0EDBCFF7FF97
:10455000100EDBCFF8FF0800F550DF6EDF5014E0DF
:10456000DEEC26F011E2EDEC26F003E1151C01E192
:10457000BCD2BBDB01E3DB2A090EDB2AD9500E0FCC
:10458000E96E000ECBDBE7D7D3DA01E1B4D2ADD2CE
:10459000C6DA110EEECFDBFF120EEDCFDBFF110EF0
:1045A000DBCFE6FF120EDBCFE6FF31EC2CF0E5525D
:1045B000E552130EF3CFDBFF140EF4CFDBFF060E34
:1045C000DB5004E0130ED0DB01E20EDBD8EC26F06A
:1045D00002E2130EDBDAAFDB05E0040EC5DB02E21C
:1045E000050ED4DA030EDBB005D0A2DA01E07DD2ED
:1045F000080EDB6A090EDB6A110EDBCFE9FF120E33
:10460000DBCFEAFFEFCFDFFFDF5014E0D7DB12E2B2
:10461000E4DB03E1151C01E168D267DB01E3DB2A7F
:10462000090EDB2A110EDB2ADBCFE9FF120EE8E3CD
:10463000DB2AE6D77DDA01E15ED257D2030EDB8EAC
:10464000070EDB0410E195DB040E5ADB0A0EEECFF9
:10465000DBFF0B0EEECFDBFF0C0EEECFDBFF0D0E04
:10466000EECFDBFF6CD0070EDB5003082CE1030E0E
:10467000DBAE0DD0B2DA020E76DAEFCF14F0156AA7
:10468000166A176A14AE39D01568166835D0F70E59
:10469000DBCF15F0F80EDBCF16F0020E155E000E24
:1046A000165AF70E15C0DBFFF80E16C0DBFF15C05B
:1046B000E9FF16C0EAFFEFCF14F00A0E14C0DBFFCB
:1046C0000B0EDB6A38D0070EDB50020809E1030E3F
:1046D000DBAE04D059DB16AE10D00ED055DB0DD0BA
:1046E000030EDBAE12D079DA020E3DDAF9DA166A81
:1046F000176A15AE02D016681768E2DA0C0E16C0FB
:10470000DBFF0D0E17C0DBFF1AD0F70EDBCF16F064
:10471000F80EDBCF17F0020E165E000E175AF70EDA
:1047200016C0DBFFF80E17C0DBFF16C0E9FF17C08D
:10473000EAFFD6DAC5DA0C0EDB6A0D0EDB6A060E6E
:10474000DB5005E1010EF36E050EF3CFDBFF150E16
:10475000DB6A160EDB6AD950370F146E000EDA20B2
:10476000156E390E14C0DBFF3A0E15C0DBFF380E94
:10477000DB6A080EDB6A0A0EAEDADF50780A12E056
:10478000200A10E0280A0CE0200A0AE03F0A06E0AE
:104790000D0A02E0200A08E1020E05D0080E03D03F
:1047A000080EDF26100E97DA030EDBBE02D0DB9276
:1047B000DB94DB50800B24E08ADAD890030EEB50B8
:1047C000000A08E6000EEE5C000EEE58000EEE58F1
:1047D000000EEE5815E213DA0B680C680D680E68CF
:1047E000F9EC34F00A0E02C0DBFF0B0E03C0DBFF56
:1047F0000C0E04C0DBFF0D0E05C0DBFF2D0E08D034
:10480000030EDBA202D02B0E03D0DBA408D0200EB7
:10481000F36E170EF3CFDBFF150EDB2A02D0170E57
:10482000DB6A050EDB5003E1B7D901E189D0EA0E5E
:10483000146E6B0E156E000E166E070EDBCF17F0A2
:10484000186A196A1A6A17C00BF018C00CF019C060
:104850000DF01AC00EF0D3D958EC35F014500224E4
:10486000F36E15500320F46E16500420F86EF4CF4A
:10487000F7FFF3CFF6FF0800090EF5CFDBFF580E68
:10488000DF5C0FE1610EF36E090E7BD90AE3200EA7
:10489000146E090EDBCFE7FF1450E75E090EE7CF79
:1048A000DBFF070EDBCF14F0156A166A176A0FDA02
:1048B00014C00BF015C00CF016C00DF017C00EF0B0
:1048C000EECF06F0EECF07F0EECF08F0EFCF09F015
:1048D00058EC35F009C0EDFF08C0EDFF07C0EDFF53
:1048E00006C0EFFF390EDBCFE9FFDB063A0EDBCF68
:1048F000EAFF01E2DB06090EDBCFEFFF150EDB2A34
:104900004BD995E1030EDBA61DD06F0EDF5C06E1EF
:10491000C1D918E3150EDB285BDA14D0780EDF5C02
:1049200009E0580EDF5C06E0620EDF5C03E0420E39
:10493000DF5C08E1020EF36E160EF3CFDBFF02D050
:10494000150EDB6A030EDB50100B0EE0040EDBCFFE
:1049500014F0050EDB50D880145406E2060EDB502E
:1049600003E1040EDB5034DA95D90AE2050EDBCF01
:10497000E7FF150EDB50E75E050EE7CFDBFF02D049
:10498000050EDB6A040EDBCF14F0160E45D9D88075
:10499000145414E2160EDBCFE6FF150EDBCFE6FF54
:1049A000040EDBCFE6FF050EDB50E552E75CE55277
:1049B000D880E754E552D880E7545FD9030EDB5026
:1049C000010B0BE1080EDB5008E0B2D801E08DD0FE
:1049D000080EDB50BED8080EDB6A170EDB5007E06E
:1049E00088D9170EF1D903E1151C01E17ED0160E0E
:1049F000DB5016E07ED9300EE66E9FD802E1151C22
:104A000074E077D9DFCFE6FFB7EC34F0E552E5523A
:104A1000E552F4CF15F00001F31C02E1151C65E02E
:104A2000050EDBCF14F0160EDB50D880145409E2CB
:104A3000050EDBCFE7FF160EDB50E75E050EE7CF76
:104A4000DBFF300EE66E050ECBD94FE1390EDB2AC7
:104A5000DBCFE9FF3A0E01E3DB2ADBCFEAFF090EE9
:104A6000EFCFDBFFDB500EE044D9090EADD902E1F8
:104A7000151C3BE0390EDB2ADBCFE9FF3A0EEDE3F4
:104A8000DB2AEBD755D831E1160EDBCFE6FF080E57
:104A9000C3D8E552E7245DD82ED0070EDB50030AB9
:104AA0001CE0010A14E0030A07E07BD9DBCFEEFF2C
:104AB000020EDBCFEDFF1FD0F5D8196A17AE02D07A
:104AC000186819682CD8BCD819C0EEFF14D0EAD8E1
:104AD00017BE186824D8B4D80ED063D9DBCFEFFF47
:104AE0000AD07BD905E1151C03E1F368F46810D006
:104AF000FCD801E3DB2A79D91AEF21F0010EDBCFD4
:104B000014F0020EDBCF15F014C0F3FF15C0F4FF54
:104B10003B0EE15C02E2E16AE552E16ECBD029D9BD
:104B2000020E80EF26F061D90800F550DF6E12000A
:104B3000200EE66E080EF0EF26F0B7EC34F0E552EA
:104B4000E552E552F3CF14F0F4CF15F00001F31C59
:104B50001200146E156AD950010F4DD91450EE266B
:104B60001550ED221200185E000E195AF70E18C0EB
:104B7000DBFFF80E19C0DBFF18C0E9FF19C0EAFF20
:104B80001200DBCFF4FFF350F45C1200DB50E76E51
:104B9000040EE7CFDBFF12000A0EDBCF14F00B0E82
:104BA000DBCF15F00C0EDBCF16F00D0EDBCF17F0C0
:104BB00014501510161017101200130EEECFDBFF55
:104BC000140EEDCFDBFF130EDBCF14F0140EDBCF92
:104BD00015F00001800E15141200F70EDBCF18F04F
:104BE000F80EDBCF19F01200050EDB50E66ED9503F
:104BF000130F01D9E552E750EE6EED6A12000A0E6E
:104C0000DBCF06F00B0EDBCF07F00C0EDBCF08F08E
:104C10000D0EDBCF09F01200DBCFE6FF150EDBCF68
:104C2000E6FF050EDB50E552E724E552E7241200CB
:104C3000DB50CED8010EF36E060EF3CFDBFF120071
:104C4000EE50EFCFEAFFE96E16C0EEFF17C0EEFFA1
:104C500018C0EEFF1200D9CFE6FFDACFE6FFE1CFB2
:104C6000D9FFE2CFDAFF1200DFCFE6FFE66A31ECD0
:104C700035F0E552E552F3501200E76E080EE7CF2B
:104C8000DBFF1200EECF14F0EECF15F0EFCF16F0F1
:104C9000176A1200050EDBCF14F0150EDB50D8801A
:104CA00014541200010EDBCF16F0020EDBCF17F00A
:104CB000186A1200E552E5CFDAFFE7CFD9FF1200FC
:104CC0000A0E14C0DBFF0B0E15C0DBFF1200D9501B
:104CD0000A0FFBEF26F0F36E070EF3CFDBFF120097
:104CE000EECF14F0EFCF15F01200010EDB2A020E0A
:104CF0001200FC0EDBCFE6FFFD0EDBCFE6FF12005D
:104D0000145E000E155AF70E14C0DBFFF80E15C026
:104D1000DBFF14C0E9FF15C0EAFF1200DA20EA6EDB
:104D2000EF2AEECFF6FF000EEF22EECFF7FFEF22D5
:104D3000EECFF8FF1200040EDBCFE6FF130EDB50C0
:104D4000E552E75C9ADFDB5004DF060EDB50120011
:104D5000090EDB500A0DF350DF24D00FE76E090E69
:104D6000E7CFDBFF93EF25F0DB50F36E050EC1EFCD
:104D700025F0F70EDBCF14F0F80EDBCF15F01200A4
:104D8000DFCFE6FF9DEF25F028DF030EECDE42EFDC
:104D900026F0EFEC20F0E552E552E552E55200092D
:104DA0001200BDDEEE50EFCFEAFFE96E010E1200F9
:104DB000130EDB50F36E040EC1EF25F0040EDB5032
:104DC000F36E090EC1EF25F0DBCFE6FF9DEF25F076
:104DD000E76E050EE7CFDBFF12008BDFC0EF26F09A
:104DE000DBCFE6FF86DFC9EF26F0D950F90FE96E79
:104DF000FF0E8EEF26F0E96E000EDA20EA6E12004A
:104E000028632920436F7079726967687420536939
:104E10006572726120526164696F205379737465A1
:104E20006D732C204C4C4300012A310101680101B3
:104E30000101012D010101010101016801010122AE
:104E400001010101010101010101010168010101EB
:104E50002D01012A73616A293F3E3C38302021230D
:104E6000272F01010131014C560611150902140BBF
:104E700010041E0D1207050F161B0A08030C180E4E
:104E8000191D1301010122010CCF2A1E0000000090
:104E9000000CB11F1E00000000000CCF2A0A000009
:104EA0000CB11F1E00000000000CCF2A0A00000CED
:104EB000CF2A0A00000CCF2A1E000000000010B10B
:104EC0001F10000010B11F1E000000000010B11FD5
:104ED00010000010B11F1E000010B11F10000010C4
:104EE000B11F1E000000000014B11F14000014B117
:104EF0001F1E000000000014B11F14000014B11F99
:104F00001E000014B11F14000014B11F1E00000089
:104F1000000010950C10000010950C1E0000000001
:104F20000010B11F10000010B11F1E000000000093
:104F300010950C10000010950C1E000010950C1020
:104F4000000010950C1E000000000010B11F1000A2
:104F50000010B11F1E000010B11F10000010B11F83
:104F60001E000000000010950C10000010950C10A1
:104F7000000010950C1E000000000010B11F100072
:104F80000010B11F10000010B11F1E000000000033
:104F90000C45121E00000000000CCF2A0A00000C75
:104FA00045121E0000000000000000145A121400F8
:104FB00000145A12140000145A12C80000C800004D
:104FC00000010064BB0F645A1200010014AB181EEC
:104FD00000000000001406231E0000000000102D39
:104FE00009100000102D091E000000000010890BA0
:104FF00010000010890B1E0000000000C82D0900E1
:105000000100C8890B000100102D09100000102DAF
:1050100009100000102D091E000000000010890B6F
:1050200010000010890B10000010890B1E000000FA
:10503000000064950C6400000001006441106400ED
:1050400000000100C8E71800010014E71814000070
:1050500014E7183C00000001000AE71846000000B1
:1050600001000AE7180A00000AE71896000000018C
:10507000000AE7181E00000001000AE7180A0000F5
:105080000AE7181E00000001000AE71832000000BD
:1050900001000AE7180A00000AE7183200000001C0
:1050A000000AE7181E00000AE7183200000001009D
:1050B0000AE7182800000001000A912C0A00000AE3
:1050C000912C0A00000A912C0A00000A912C0A0077
:1050D000000A912C0A00000000000A0D370A0000A7
:1050E0000A0D370A00000A0D370A00000A0D370AB8
:1050F00000000A0D370A0000000000140D3714915B
:105100002C140D3714912C140D3714912C140D37C9
:1051100014912C140D3714912C0000000000001481
:105120000D3714912C140D3714912C140D37149144
:105130002C140D3714912C140D3714912C140D3799
:1051400014912C140D3714912C140D37000000000D
:10515000000014950C14000014950C140000149514
:105160000C14000014950C14000014950C1400008D
:10517000000000146B0E140000146B0E14000014D9
:105180006B0E140000146B0E140000146B0E140050
:105190000000000014950C146B0E14950C146B0E8B
:1051A00014950C146B0E14950C146B0E14950C14B2
:1051B0006B0E000000C87C0A00010020950C100056
:1051C0000010950C1E000000000010000020B11F10
:1051D00030000000000027F9140D00000DF914271D
:1051E000000027F9140D000027F9140D000027F91D
:1051F000142700000000000DF9142700000DF91419
:105200000D000027F9140D00000DF9142700000D02
:10521000F9140D000027F9140D00000DF9142700F2
:105220000000000027F9140D00000DF914270000FC
:105230000DF9140D000027F914270000000000A844
:105240004F000000000030001830003030004830BF
:1052500000603000783000903000A83000C030008E
:10526000D83000F0300008310020310038310050D3
:105270003100683100803100983100B03100C83110
:1052800000E03100F83100103200283200403200D6
:10529000583200703200883200A03200B83200D09C
:1052A0003200E83200884E000000009A4E000000F4
:1052B00000904F00000000BE4E00000000914E0024
:1052C000000000AB4F00000000C34F00000000CC06
:1052D0004F00D54F00DE4F00ED4F00FC4F00025055
:1052E000003250003B5000994F0000000044500035
:1052F0000000004A50000000005950000000006209
:105300005000000000CD4E00000000B95000DA50FF
:10531000005251007351000850001D5000A94E006A
:10532000000000B551000000007150000000007A3C
:105330005000000000E84E00000000F74E000000A2
:1053400000124F00214F00304F004B4F00664F00BE
:105350007B4F00BB5100CA510089500000000092F1
:105360005000000000FB50000000009451000000BD
:1053700000A15000000000D65100000000F75100CD
:10538000000000B050000000002452000000001F88
:0D5390005100000000080C101418202864C3
:02539E009D98D8
:1053A0009D9ACAD80001E86B949C948E9F9A9F980E
:1053B000240EAC6E900EAB6EB886800EE66E250E97
:1053C000E66EE66AE66A3AD85CEF2BF09D989D9A05
:1053D000AB9E120061D9186A2D0E196E310E1A6E2D
:1053E000010E1B6E18C006F019C007F01AC008F0B5
:1053F000096EFB0EDBCF0BF0FC0EDBCF0CF0FD0ECD
:10540000DBCF0DF0FE0EDBCF0EF058EC35F006C012
:1054100014F007C015F008C016F009C017F0140604
:10542000000E155A165A175AD890173216321532DE
:10543000143214C0F3FF15C0F4FF33D12DD9030E7D
:10544000E126D950FB0FE96EFF0EDA20EA6EEECFAF
:10545000E6FFEECFE6FFEECFE6FFEFCFE6FFBADFE7
:105460002BD9F3CFDEFFF4CFDDFF9D50200B03E1FE
:105470009D50100B06E0010EF36E020EF3CFDBFF22
:1054800002D0020EDB6A9D989D9ADECF14F0DDCF2C
:1054900015F015C014F0156A1450B06EDF50AF6EE1
:1054A000020EDB5002E09D889D8A030EE15C02E261
:1054B000E16AE552E16EF5D09E50100B05E09D507B
:1054C000100B02E00AD8010C9E50200B05E09D5005
:1054D000200B02E010D8010C000CDED8E65207D9F0
:1054E00076D8E552E552000903E0DF50AD6E01D0F9
:1054F0009D98E552D6D0D0D8E652ABA203D0AB9857
:10550000AB880BD0AE50DF6EABB407D0DFCFE6FF79
:10551000F30EE66E000EDDD802D00001E881E55200
:10552000C0D0EAD801E1000C010CE6D803E1F25149
:10553000010B01E1000C010C320EE66E000EE66E6E
:10554000030EE66EF30EE66E000EBBD8640EE66E3A
:10555000000EE66E0F0EE66EED0EE66E000E61EFCB
:105560002BF09AD89D9AA1D8F30EE66E000EE66E47
:105570003EEC33F0A1D8000903E09D8A010E02D071
:105580009D8A000E8ED088D80001F8B113D0F75153
:10559000EA6AF325E96EF451EA22EF50E66EFD0E59
:1055A000DBCFE9FFFE0EDBCFEAFFE552E750EF6EFF
:1055B000010E01D0000E75D06FD89D98FE0EDBCF86
:1055C000E6FFED0EE66E000E84D89D886AD064D8A2
:1055D0006CD8ED0EE66E000EE66E3EEC33F06CD845
:1055E00060D05AD889D80DE17BD85FD831EC2CF047
:1055F000E552E552F3CFEBF0F4CFECF013D8010E07
:1056000001D0000E4ED048D877D80AE169D8FB0EF9
:10561000DBCFEBF0FC0EDBCFECF004D8010E01D0B9
:10562000000E3FD069D81BE0EB51EC1113E0F251B2
:10563000020B10E1E9C0E9FFEAC0EAFFE92B000E26
:10564000EA23EF50E66EB8DFE5520001EB07000EEB
:10565000EC5BEAD7EB51EC1102E1E96BEA6B12006B
:105660000001E96BEA6B9CEF2AF016D8E6520001C4
:10567000F8B110D03CD887DFE552E552DFCFE6FF26
:105680002EEC01F0E552000905E131D86ADFE55260
:10569000E552EDD7E55205D0D9CFE6FFE1CFD9FFEE
:1056A0001200E552E7CFD9FF1200FD0EDBCFE6FF77
:1056B000FE0EDBCFE6FF1200E552E552E552E55261
:1056C0001200E66E08EC33F0146E050EE15E145025
:1056D0001200E66E22EC33F0E552E552E55212007C
:1056E000FD0EDBCFE9F0FE0EDBCFEAF01200D9CFE2
:1056F000E6FFDACFE6FF12000001E951EA111200DD
:10570000D9CFE6FFDACFE6FFFA0EE3CFD9FFFB0EE3
:10571000E3CFDAFFFC0EE3CFE9FFFD0EE3CFEAFFB4
:10572000E9CFF3FFEACFF4FFF80EE35003E1F90EFF
:10573000E35008E0F80EE30602E2F90EE306DECFDE
:10574000EEFFF2D7FF0EE3CFDAFFE552FF0EE3CF15
:10575000D9FFE5521200D9CFE6FFDACFE6FFFA0E05
:10576000E3CFD9FFFB0EE3CFDAFFFC0EE3CFE9FF77
:10577000FD0EE3CFEAFFE9CFF3FFEACFF4FFE950F4
:10578000D95CEA50DA580EE3F80EE35003E1F90E63
:10579000E35024E0F80EE30602E2F90EE306DECF62
:1057A000EEFFF2D7F80EE350D926F90EE350DA22D5
:1057B000DD52F80EE350E926F90EE350EA22ED52ED
:1057C000F80EE35003E1F90EE35008E0F80EE306AB
:1057D00002E2F90EE306DDCFEDFFF2D7FF0EE3CFD5
:1057E000DAFFE552FF0EE3CFD9FFE5521200D9CF21
:1057F000E6FFDACFE6FFFA0EE3CFD9FFFB0EE3CFE9
:10580000DAFFFC0EE3CFE9FFFD0EE3CFEAFFE9CFBD
:10581000F3FFEACFF4FFDECFEFFFEE66FCD7FF0E1B
:10582000E3CFDAFFE552FF0EE3CFD9FFE5521200D6
:10583000FB0EE3CFF6FFFC0EE3CFF7FFFD0EE3CF49
:10584000F8FFFE0EE3CFE9FFFF0EE3CFEAFFE9CF5B
:10585000F3FFEACFF4FF0900F5CFEFFFEE66FBD7C9
:105860001200FE0EE3CFE9FFFF0EE3CFEAFFF36A7B
:10587000F46AEE5203E0F34AF42AFBD71200FF0E5B
:10588000E3CFF8FFE552FF0EE3CFF7FFE552FF0E3F
:10589000E3CFF6FFE552E66AE66AE66A0900F552EA
:1058A00009E0FD0EE32A05E1FE0EE32A02E1FF0E08
:1058B000E32AF4D7FD0EE3CF07F0FE0EE3CF08F0A6
:1058C000FF0EE3CF09F01200D9CFE6FFDACFE6FFF3
:1058D000FA0EE3CFD9FFFB0EE3CFDAFFFC0EE3CFE6
:1058E000E9FFFD0EE3CFEAFFE9CFF3FFEACFF4FFD4
:1058F000F80EE35003E1F90EE3500BE0F80EE30677
:1059000002E2F90EE306DECFEFFFEE66F1D7DD52DD
:10591000EFD7FF0EE3CFDAFFE552FF0EE3CFD9FF5B
:10592000E5521200FB0EE3CFF6FFFC0EE3CFF7FFCC
:10593000FD0EE3CFF8FFFE0EE3CFE9FFFF0EE3CF4E
:10594000EAFFE9CFF3FFEACFF4FFF90EE35003E1FA
:10595000FA0EE3500CE0F90EE30602E2FA0EE3065B
:105960000900F5CFEFFFEE66F0D70A00EED7120080
:10597000FE0EE3CFE9FFFF0EE3CFEAFFF36AF46A1E
:10598000FD0EE350EF5C04E1E9CFF3FFEACFF4FF53
:06599000EE66F6D71200DE
:0A5996009EB09DA001D002D0000ECB
:1059A00012000E01F6CF1FFEF7CF20FEF8CF21FE2A
:1059B000F5CF22FEF3CF23FEF4CF24FEE9CF25FE60
:1059C000EACF26FED9CF27FEDACF28FE550EF29E6B
:1059D000CE5C2D6FC30ECF5A2DCECEFFF28E29672F
:1059E00029072A672A072B672B072C672C073C6798
:1059F0003C073D673D073E673E075C675C07352F08
:105A000002D0140E356F3F2F07D0C80E3F6FE86AE3
:105A1000402B41234223432336A12CD029672AD08F
:105A200036A505D037CE29FE119D369523D0466781
:105A300011D044CEE9FF45CEEAFFEFCF46FE4667E0
:105A400001D017D0444B452B010E466303D03ACE0C
:105A500029FE10D0D890463309E003E237CE29FE64
:105A600002D039CE29FE118D368504D038CE29FEDC
:105A700001D0369136A93CD02A673AD047CEE9FF0B
:105A800048CEEAFF030E4727E86A4823EE5027E096
:105A90002A6FEECF2FFEEE50306F03E12F5101E160
:105AA0001CD05B5110E02F3530359D0D5751F4025D
:105AB000F336F43406E2F336E83403E2F336E8343E
:105AC00003E3FF0E01D057519D921A6F2FCE12FEA5
:105AD00030CE13FE9D8211810BD0119109D0EE5072
:105AE00005E04FCE47FE50CE48FE02D036991191C8
:105AF00036AB3CD02B673AD049CEE9FF4ACEEAFF1D
:105B0000030E4927E86A4A23EE5027E02B6FEECFB9
:105B100031FEEE50326F03E1315101E11CD05B5197
:105B200010E0313532359D0D5851F402F336F4341E
:105B300006E2F336E83403E2F336E83403E3FF0E1B
:105B400001D058519D921B6F31CE14FE32CE15FEFE
:105B50009D8211850BD0119509D0EE5005E051CEF4
:105B600049FE52CE4AFE02D0369B119536AD3CD04E
:105B70002C673AD04BCEE9FF4CCEEAFF030E4B2701
:105B8000E86A4C23EE5027E02C6FEECF33FEEE5048
:105B9000346F03E1335101E11CD05B5110E0333528
:105BA00034359D0D5951F402F336F43406E2F336E0
:105BB000E83403E2F336E83403E3FF0E01D0595131
:105BC0009D921C6F33CE16FE34CE17FE9D82118936
:105BD0000BD0119909D0EE5005E053CE4BFE54CEB8
:105BE0004CFE02D0369D119928CEDAFF27CED9FF80
:105BF00026CEEAFF25CEE9FF24CEF4FF23CEF3FF25
:105C000022CEF5FF21CEF8FF20CEF7FF1FCEF6FF04
:065C10009E90010E12003F
:0A5C160027D9E65294869488160EF2
:105C2000C66E010EC56EFE0EDB50E824C86EC76A54
:105C3000FC0EDBCFDFF2FD0EDBCFE0F2FA0EDBCFA6
:105C4000E1F2FB0EDBCFE2F2F90EDB040201E36FBF
:105C5000F70EDBCFE4F2F80EDBCFE5F2F50EDBCF8B
:105C6000E6F2F60EDBCFE7F2C68A9E96E552E552E3
:105C7000E7CFD9FF1200F7D8020EE126010EDB6A4A
:105C80009EA648D0C69C2D0EC714090A1EE0050A20
:105C900002E0010A37E1C950DF6E9E96E4C2E6FFDA
:105CA000E5C2E6FFE6C2E9FFE7C2EAFFEF50E66EB3
:105CB0003AD8E552E552E552DF6EE6C2E9FFE7C2A7
:105CC000EAFFEF6ADF5017E11AD0C950DF6E9E96E7
:105CD000C688E3C2E6FFDFC2E6FFE0C2E6FFE1C23C
:105CE000E6FFE2C2E6FF5AD8146E050EE15E1450DC
:105CF000DF6EDF5004E0010EDFCFDBFF0BD0010EC3
:105D0000DB6808D0C950DF6E9E96C69CC688DE52FE
:105D1000050EDD6E010EDB50146E020EE15C02E238
:105D2000E16AE55291D09FD8030EE1260E013C694D
:105D3000FE0EDB50C96E9E96C688FC0EDBCF08F0C7
:105D4000FD0E88D8FE0EDB50DF6EDF501FE09E5048
:105D5000080B02E13C51FBE13C5102E1010E17D07E
:105D60002D0EC7142C0A07E0040A04E09E96C6888C
:105D7000020E0DD0DF6ADF5005E07AD801E3DB2A9E
:105D8000EF50C96E9E96C688DF06DFD7000E146EF0
:105D9000030EE15C02E2E16AE55256D064D8050EDA
:105DA000E1260E013C696CD8EF6A9E50080B02E1B7
:105DB0003C51FBE13C512BE02D0EC714290A2DE18B
:105DC000040EC9CFDBFF9E96C688FB0EDBCF08F022
:105DD000FC0E40D8040EDB50F36EFA0EDBCFF4FF5E
:105DE000F350F45C06E2FA0EDB50E76E040EE7CFE8
:105DF000DBFF040EDB50DF6EDF501EE09E50080B11
:105E000003E10E013C51FAE10E013C5102E1010EA9
:105E100014D02D0EC714290A04E09E96C688020EDF
:105E20000CD09E96C68824D801E3DB2AC9CFEFFFA9
:105E300027D8EF2ADF06E0D7000E146E050EE15CCE
:105E400002E2E16AE55200D0E16E1450E552E7CF7C
:105E5000D9FF1200DBCF09F0DE5208C0DEFF09C017
:105E6000DDFFDD521200D9CFE6FFE1CFD9FF1200EE
:105E7000010EDBCFE9FFDB2A020EDBCFEAFF1200C7
:0E5E8000FD0EDBCFE9FFFE0EDBCFEAFF1200C6
:025E8E0040775B
:105E90001B0080841E00A0252600A0252600E067A8
:105EA000350000093D00404B4C00404B4C0044562F
:105EB000510044565100C4945100C4945100E4E28E
:105EC0005100E4E251006CF65100AE0452006C73D4
:105ED00052006C735200C0CF6A00A0636F008096BE
:105EE000980080969800201D9A0070E09A00809F8C
:105EF000D500B0F6DA00C0E1E400C0E1E40020B271
:105F00001301C0381501406F4001104D470190CA80
:105F10007B0130517D01003FAB01A02FC50180F016
:105F2000FA0280F9370300449508004DD2080007B3
:105F3000AE09F050B00980733B0D403A690D00B1D5
:105F400008198074D21A806DC3350028503700E6D6
:105F5000E849006D7C4D00000000000000000000DA
:105F60000000000000000000000000000000000031
:105F70000000000000000000000000000000000021
:105F80000000000000000000000000000000A0254C
:105F90002600A0252600E067350080EE3600404B45
:105FA0004C00404B4C00C0CF6A0008B86C00809693
:105FB000980080969800201D9A0070E09A00809FBB
:105FC000D50070E9D700C0E1E400C0E1E40020B2F0
:105FD000130130561401406F4001807C430190CA88
:105FE0007B01D0667C01003FAB01E0D2AF0180F0C5
:105FF000FA022077FC0200449508A0CA9608000720
:10600000AE09F050B00900000000000000000000E0
:106010000000000000000000000000000000000080
:106020000000000000000000000000000000000070
:106030000000000000000000000000000000000060
:106040000000000000000000000000000000000050
:106050000000000000000000000000000000000040
:106060000000000000000000000000000000000030
:106070000000000000000000000000000000000020
:0E608000000000000000000000000000000012
:02608E000E0101
:10609000F6CF00FEF7CF01FEF8CF02FEF5CF03FEEC
:1060A000F3CF04FEF4CF05FE0E6B106B12510627E2
:1060B00013510723145108271551092311B101D099
:1060C00020D011A305D01ECE0EFE07BF0E6D11D03D
:1060D000000EF86E07517F0BF66E800EF6262F0E1F
:1060E000F76E02E3F74AF82A0800F55007BFE86C9C
:1060F0000E6F1A510E030EBFF45EF3CF10FEF4CFF5
:106100000EFE11A520D011A705D01ECE0FFE09BF8F
:106110000F6D11D0000EF86E09517F0BF66E800ED8
:10612000F6262F0EF76E02E3F74AF82A0800F5501C
:1061300009BFE86C0F6F1B510F030FBFF45EF350E4
:106140001027F4500E231051800FE86A0E23800EA2
:106150000E25BE6E0E6B106B16510A2717510B23BE
:1061600018510C2719510D2311B901D020D011ABB2
:1061700005D01ECE0EFE0BBF0E6D11D0000EF86EB8
:106180000B517F0BF66E800EF6262F0EF76E02E394
:10619000F74AF82A0800F5500BBFE86C0E6F1C5147
:1061A0000E030EBFF45EF3CF10FEF4CF0EFE11AD62
:1061B00020D011AF05D01ECE0FFE0DBF0F6D11D038
:1061C000000EF86E0D517F0BF66E800EF6262F0E28
:1061D000F76E02E3F74AF82A0800F5500DBFE86CA5
:1061E0000F6F1D510F030FBFF45EF3501027F450D3
:1061F0000E231051800FE86A0E23800E0E25BB6E11
:106200009E9205CEF4FF04CEF3FF03CEF5FF02CE3F
:0C621000F8FF01CEF7FF00CEF6FF1200F1
:04621C00FF0EE3CFBF
:10622000EAFFE552FF0EE3CFE9FFE552E66AE66AD0
:10623000E66AE66AD9CFE6FFDACFE6FFFA0EE12496
:10624000D96EFF0EE220DA6EE66AE66AE66AE66A70
:10625000E66A200EEF5C06E0090EEF5C03E0EF66F5
:1062600003D06BD0EE50F5D72D0EEF5C03E1FF0E9F
:10627000E32A03D02B0EEF5C01E1EE502F0EEF640A
:1062800044D03A0EEF6041D0D890F50EE336F60ECA
:10629000E336F70EE336F80EE336FB0EDECFE3FF10
:1062A000FC0EDECFE3FFFD0EDECFE3FFFE0EDDCF03
:1062B000E3FFDD52DD52D890F50EE336F60EE336FD
:1062C000F70EE336F80EE336D890F50EE336F60E09
:1062D000E336F70EE336F80EE336FB0EE350DE2628
:1062E000FC0EE350DE22FD0EE350DE22FE0EE350F4
:1062F000DD22DD52DD52300EEE5CDE26000EDE22A7
:10630000DE22DD22DD52DD52B9D7FF0EE3CFE8FFFA
:10631000E85213E0F50EE31EF60EE31EF70EE31E41
:10632000F80EE31EF50EE32A08E1F60EE32A05E176
:10633000F70EE32A02E1F80EE32AE552E552E552B0
:10634000E552E552D9CFE9FFDACFEAFFEECF06F00A
:10635000EECF07F0EECF08F0EFCF09F0FF0EE3CF5E
:10636000DAFFE552FF0EE3CFD9FFE552E552E552E1
:02637000120019
:0E6372008DD8F8CFE4FFF5CFE4FFE65247ECFC
:1063800030F0E552E5CFF5FFE5CFF8FF8ED07FD8AE
:10639000F6CFE4FFF7CFE4FFF8CFE4FFF5CFE4FF5B
:1063A000F3CFE4FFF4CFE4FFFACFE4FFFBCFE4FF49
:1063B00000EE00F0140EE80403E3EECFE4FFFBD799
:1063C00000EE14F0120EE80403E3EECFE4FFFBD777
:1063D000E6525CEC2AF0000902E1CBEC2CF0E5522D
:1063E00000EE25F0120EE80403E3E5CFEDFFFBD746
:1063F00000EE13F0140EE80403E3E5CFEDFFFBD746
:10640000E5CFFBFFE5CFFAFFE5CFF4FFE5CFF3FFE4
:10641000E5CFF5FFE5CFF8FFE5CFF7FFE5CFF6FFD6
:1064200044D0D9CFE6FFE1CFD9FF240EE12684EC9A
:1064300011F09D829D80F28EF28C0E01010E3B6F59
:106440009D889D8A0400ECEC15F0146814C0E6FFEA
:106450003BEC2EF0E552E7CF14F0DF6E145C02E166
:106460007DEC12F012EC1AF08FEC1AF012EC2BF01B
:1064700035EC2BF030EC00F0E5D7240EE15C02E2C5
:10648000E16AE552E16EE552E7CFD9FF1200D8CFBD
:10649000E4FFE0CFE4FFE46EDACFE4FFE2CFDAFF1F
:1064A000E9CFE4FFEACFE4FF1200E5CFEAFFE5CF52
:1064B000E9FFE5CFDAFFE550E5CFE0FFE5CFD8FF14
:0264C0001000CA
:0E64C200D9CFE6FFE1CFD9FF020EE12600019F
:1064D000F96BFA6BFB6BFC6BD950FC0FE96EFF0E8E
:1064E000DA20EA6EEFCFF6FF020EEE26EFCFF7FFCF
:1064F000000EEE22EFCFF8FF000EEE220900F5CFDE
:10650000FBF00A00F5CFFCF0FA0EDB06FB0E01E211
:10651000DB06FA0EDBCF14F0DB06FB0EDBCF15F04B
:1065200001E2DB06145015103FE00400D950FC0FC7
:10653000E96EFF0EDA20EA6EEFCFF6FF020EEE26CE
:10654000EFCFF7FF000EEE22EFCFF8FF000EEE22A6
:106550000900F5CFF9F00A00F5CFFAF0100EDE6E63
:10656000DD6AD9CFE9FFDACFEAFFEE50ED101BE08C
:106570000001FB51800B0CE00001D890F937FA378D
:10658000FB37FC37210E0001FB1B0001FC7706D016
:106590000001D890F937FA37FB37FC37DF06010ED8
:1065A00001E2DB06DED7B5D7200EDE6EDD6AD9CF7D
:1065B000E9FFDACFEAFFEE50ED101BE00001FB51DE
:1065C000800B0CE00001D890F937FA37FB37FC3725
:1065D000210E0001FB1B0001FC7706D00001D890C2
:1065E000F937FA37FB37FC37DF06010E01E2DB062D
:1065F000DED7FBC0F3FFFCC0F4FF00D0020EE15C6D
:1066000002E2E16AE552E16EE552E7CFD9FF1200FE
:10661000D9CFE6FFE1CFD9FF55D8FB0EDBCFEEFF98
:10662000FC0EDBCFEDFF4ED8020E53D8FA0EDBCFB7
:10663000EFFF60D8EF925ED8EF8060D8EF6A62D843
:10664000EF6A54D072D8020B17E158D867D8FC0E05
:10665000DBCFEFFF4FD8EF9051D858D802E34ED898
:10666000EF6A4CD8EFCF14F04DD8EF50145C02E134
:1066700041D8EF82010E01D0000E38D056D8010B60
:106680001FE140D84BD8EF50E66EFB0EDBCFE9FFA1
:10669000FC0EDBCFEAFFE552E750EF6E2BD8EF920E
:1066A00031D834D802E32ED8EF6A2CD8EFCF14F0CB
:1066B00025D8EF50145C02E11DD8EF80010E01D007
:1066C000000E14D0FD0EDBCFE9FFFE0EDBCFEAFF9C
:1066D0001200E926000EEA2212001450EE24E76EA2
:1066E0001550EE20EA6EE7CFE9FF1200E552E7CF42
:1066F000D9FF1200E7DF050E69EF33F0E3DF030E89
:1067000069EF33F0DFDF040E69EF33F0EFCF14F001
:10671000D9DF020EDEDFEF50145C1200EF50EF2ADB
:10672000146E156ACFDF6DEF33F0D9CFE6FFE1CFFE
:08673000D9FFE0DFEF50120079
:0867380009C013F008C012F0C3
:1067400007C011F007500C02F4CF05F0F3CF04F0AE
:1067500008500D02F4CF07F0F3CF06F00C02F3500F
:106760000526F4500622E86A072211500D02F35064
:106770000526F4500622E86A072209500C02F3505D
:106780000626F450072209500D02086AE86A08221A
:10679000F3500726F450082211500E02F35006263B
:1067A000F4500722096AE86A0822092212500E02F0
:1067B000F3500726F4500822E86A092213500E020B
:1067C000F3500826F4500922000C09C013F008C049
:1067D00012F008500D02F4CF07F0F3CF06F0095085
:1067E0000E02F4CF09F0F3CF08F00D02F3500726A4
:1067F000F4500822E86A092212500E02F3500726CC
:10680000F4500822E86A09220EAE0BEF34F0125061
:10681000085E1350095A13AE000C0D50085E0E505E
:04682000095A000C05
:0C682400D9CFE6FFDACFE6FFE1CFD9FFC5
:10683000E2CFDAFFE652E652E652E652D950F90FBD
:10684000146EFF0EDA20156E020E14C0DBFF030E6D
:1068500015C0DBFF020EDBCFE6FF030EDBCFE6FF4A
:10686000F90EDBCFE6FFFA0EDBCFE6FFFB0EDBCF48
:10687000E6FFD950FC0FE66EFF0EDA20E66E05EC5F
:1068800021F0146E070EE15C02E2E16AE552E16E6E
:106890001450F3CFDEFFF4CFDDFFFC0EDBCFE9FFBA
:1068A000FD0EDBCFEAFFEF6ADECF14F0DDCF15F08F
:1068B00014C0F3FF15C0F4FF040EE15C02E2E16ACC
:1068C000E552E16EE552E5CFDAFFE7CFD9FF1200DE
:1068D0002A0EF66E000EF76E000EF86E0F0109001C
:1068E000F550696F0900F5506A6F03E1696701D0DF
:1068F0003DD00900F550646F0900F550656F09003F
:10690000F550666F09000900F550E96E0900F55071
:10691000EA6E090009000900F550676F0900F5509B
:10692000686F09000900F6CF6BFFF7CF6CFFF8CF57
:106930006DFF64CFF6FF65CFF7FF66CFF8FF0F015D
:10694000675302E1685307E00900F550EE6E6707F0
:10695000F8E26807F9D76BCFF6FF6CCFF7FF6DCF82
:0E696000F8FF0F016907000E6A5BBFD7120037
:02696E00D9CF7F
:10697000E6FFDACFE6FFE1CFD9FFE2CFDAFFFB0E89
:10698000DBCF14F0FC0EDBCF15F00001800E1514E8
:106990001AE1FB0EDBCFE9FFFC0EDBCFEAFFEECF07
:1069A000F3FFEDCFF4FFEE2A000EEF22F3CFE9FF65
:1069B000F4CFEAFFFD0EDBCFEFFFEF50156AF36E69
:1069C00015C0F4FF10D0FB0EDB50FE0806E1FD0EF3
:1069D000DBCFE6FFD9EC35F005D0FD0EDBCFE6FFCF
:1069E00005EC36F0E552E552E5CFDAFFE7CFD9FF07
:0269F000120093
:0E69F20006500B02F3CF02F0F4CF03F00C02BC
:106A0000F3500326000EF420046E06500D02F350DE
:106A10000426000EF420056E06500E02F3500526E3
:106A200007500B02F3500326F4500422000E0522F7
:106A300007500C02F3500426F450052207500D02B3
:106A4000F350052608500B02F3500426F45005229B
:106A500008500C02F350052609500B02F35005268E
:026A6000120022
:0E6A6200F36AF46AFF0EE124E96EFF0EE220F3
:106A7000EA6EED6607D02F0EEF6404D03A0EEF6099
:106A800001D0F32A1200F36AF46AFF0EE124E96EE2
:106A9000FF0EE220EA6EED660AD0200EEF5C06E003
:106AA000080EEF6404D00E0EEF6001D0F32A12003E
:106AB000056A046A036A026A200EE76ED8900636F9
:106AC00007360836093602360336043605360B50CB
:106AD000025C0C5003580D5004580E50055809E341
:106AE0000B50025E0C50035A0D50045A0E50055ABA
:086AF000062AE72EE4D712008C
:086AF800202073727330303965
:106B000038722000206E6F20696420736574200045
:106B10007031007030007430300074253264006FC2
:106B2000332530356C64006F32006F31006F3000F8
:076B3000662530356C64009E
:086B3800FF0EE350276EEF0E83
:106B400001D0F30EE76EE72EA3EF35F00C0E266EA4
:106B5000E76AE72EA9EF35F0262EA8EF35F0272EAD
:066B6000A1EF35F0120068
:0A6B6600056A046A100EE76ED8906D
:106B700008360936043605360D50045C0E500558AB
:106B800005E30D50045E0E50055A082AE72EF0D793
:026B90001200F1
:0E6B92001DEE00F02DEE00F0F86A019CFEEC06
:106BA00035F068EC34F006EC36F011EC32F0FBD73F
:026BB0001200D1
:0E6BB200FF0EE350ACBA04D0AF6AAB8EAC8AD3
:0E6BC000949CACA2FED7AD6EF36EF46A120088
:026BCE00056A56
:106BD000080EE76ED890093605360E50055C02E3C4
:0A6BE000056E092AE72EF7D7120010
:066BEA0030313233343576
:0B6BF000363738396162636465660067
:046BFC0000EE00F0B7
:0A6C00000F0EEE6AEA62FDD71200E3
:026C0A00120076
:026C0C00120074
:026C0E00000084
:036C100000000081
:0A6C13001810141014009402A502DA
:036C1D000000571D
:106C2000FFFF0000FFFF000001015D0E00000000FB
:106C30000000000000000000000000000000000054
:106C40000000000000000000000000000000000044
:106C50000000000000000000000000000000000034
:106C60000000000000000000000000000000000024
:106C70000000000000000000000000000000FEFE18
:056C800028E001010104
:020000040030CA
:0100010006F8
:0100020018E5
:010003001AE2
:010005008179
:010006008178
:00000001FF
